Microsoft (R) Macro Assembler Version 5.10                  2/14/25 23:44:19
DEBCONST.ASM                                                Page     1-1


					   PAGE    80,132 ;
					   TITLE DEBCONST.ASM
				.LIST
				.CREF
				
 0000				CODE	   SEGMENT PUBLIC BYTE
 0000				CODE	   ENDS
				
 0000				CONST	   SEGMENT PUBLIC BYTE
 0000				CONST	   ENDS
				
 0000				CSTACK	   SEGMENT STACK
 0000				CSTACK	   ENDS
				
 0000				DATA	   SEGMENT PUBLIC BYTE
 0000				DATA	   ENDS
				
				DG	   GROUP CODE,CONST,CSTACK,DATA
				
 0000				CODE	   SEGMENT PUBLIC  BYTE
				
					   EXTRN ALUFROMREG:NEAR, ALUTOREG:NEAR, ACCIMM:NEAR, SEGOP:NEAR
					   EXTRN ESPRE:NEAR, SSPRE:NEAR, CSPRE:NEAR, DSPRE:NEAR
					   EXTRN REGOP:NEAR, NOOPERANDS:NEAR, SAVHEX:NEAR, SHORTJMP:NEAR
					   EXTRN MOVSEGTO:NEAR, WORDTOALU:NEAR, MOVSEGFROM:NEAR
					   EXTRN GETADDR:NEAR, XCHGAX:NEAR, LONGJMP:NEAR, LOADACC:NEAR
					   EXTRN STOREACC:NEAR, REGIMMB:NEAR, SAV16:NEAR, MEMIMM:NEAR
					   EXTRN INT3:NEAR, SAV8:NEAR, CHK10:NEAR, M8087:NEAR
					   EXTRN M8087_D9:NEAR, M8087_DB:NEAR, M8087_DD:NEAR
					   EXTRN M8087_DF:NEAR, INFIXB:NEAR, INFIXW:NEAR, OUTFIXB:NEAR
					   EXTRN OUTFIXW:NEAR, JMPCALL:NEAR, INVARB:NEAR, INVARW:NEAR
					   EXTRN OUTVARB:NEAR, OUTVARW:NEAR, PREFIX:NEAR, IMMED:NEAR
					   EXTRN SIGNIMM:NEAR, SHIFT:NEAR, SHIFTV:NEAR, GRP1:NEAR
					   EXTRN GRP2:NEAR, REGIMMW:NEAR, DOORG:NEAR
				
				
					   EXTRN DB_OPER:NEAR, DW_OPER:NEAR, ASSEMLOOP:NEAR, GROUP2:NEAR
					   EXTRN NO_OPER:NEAR, GROUP1:NEAR, FGROUPP:NEAR, FGROUPX:NEAR
					   EXTRN FGROUPZ:NEAR, FD9_OPER:NEAR, FGROUPB:NEAR, FGROUP:NEAR
					   EXTRN FGROUPDS:NEAR, DCINC_OPER:NEAR, INT_OPER:NEAR
					   EXTRN IN_OPER:NEAR, DISP8_OPER:NEAR, JMP_OPER:NEAR, L_OPER:NEAR
					   EXTRN MOV_OPER:NEAR, OUT_OPER:NEAR, PUSH_OPER:NEAR
					   EXTRN GET_DATA16:NEAR, FGROUP3:NEAR, FGROUP3W:NEAR
					   EXTRN FDE_OPER:NEAR, ESC_OPER:NEAR, AA_OPER:NEAR
					   EXTRN CALL_OPER:NEAR, FDB_OPER:NEAR, POP_OPER:NEAR, ROTOP:NEAR
					   EXTRN TST_OPER:NEAR, EX_OPER:NEAR
				
 0000				CODE	   ENDS
				
 0000				CONST	   SEGMENT PUBLIC BYTE
				
					   PUBLIC REG8, REG16, SREG, SIZ8, DISTAB, DBMN, ADDMN, ADCMN, SUBMN
					   PUBLIC SBBMN, XORMN, ORMN, ANDMN, AAAMN, AADMN, AASMN, CALLMN, CBWMN
					   PUBLIC UPMN, DIMN, CMCMN, CMPMN, CWDMN, DAAMN, DASMN, DECMN, DIVMN
					   PUBLIC ESCMN, HLTMN, IDIVMN, IMULMN, INCMN, INTOMN, INTMN, INMN
					   PUBLIC IRETMN, JAMN, JCXZMN, JNCMN, JBEMN, JZMN, JGEMN, JGMN, JLEMN
					   PUBLIC JLMN, JMPMN, JNZMN, JPEMN, JNZMN, JPEMN, JPOMN, JNSMN, JNOMN
					   PUBLIC JOMN, JSMN, LAHFMN, LDSMN, LEAMN, LESMN, LOCKMN, LODBMN
					   PUBLIC LODWMN, LOOPNZMN, LOOPZMN, LOOPMN, MOVBMN, MOVWMN, MOVMN
					   PUBLIC MULMN, NEGMN, NOPMN, NOTMN, OUTMN, POPFMN, POPMN, PUSHFMN
					   PUBLIC PUSHMN, RCLMN, RCRMN, REPZMN, REPNZMN, RETFMN, RETMN, ROLMN
					   PUBLIC RORMN, SAHFMN, SARMN, SCABMN, SCAWMN, SHLMN, SHRMN, STCMN
					   PUBLIC DOWNMN, EIMN, STOBMN, STOWMN, TESTMN, WAITMN, XCHGMN, XLATMN
					   PUBLIC ESSEGMN, CSSEGMN, SSSEGMN, DSSEGMN, BADMN
				
					   PUBLIC M8087_TAB, FI_TAB, SIZE_TAB, MD9_TAB, MD9_TAB2, MDB_TAB
					   PUBLIC MDB_TAB2, MDD_TAB, MDD_TAB2, MDF_TAB, OPTAB, MAXOP, SHFTAB
					   PUBLIC IMMTAB, GRP1TAB, GRP2TAB, SEGTAB, REGTAB, REGTABEND, FLAGTAB
					   PUBLIC STACK
				
					   PUBLIC AXSAVE, BXSAVE, CXSAVE, DXSAVE, BPSAVE, SPSAVE, SISAVE
					   PUBLIC DISAVE, DSSAVE, ESSAVE, SSSAVE, CSSAVE, IPSAVE, FLSAVE, RSTACK
					   PUBLIC REGDIF, RDFLG, TOTREG, DSIZ, NOREGL, DISPB, LBUFSIZ, LBUFFCNT
					   PUBLIC LINEBUF, PFLAG, COLPOS, RSETFLAG
				
				
Microsoft (R) Macro Assembler Version 5.10                  2/14/25 23:44:19
DEBCONST.ASM                                                Page     1-2
                                                            

					   PUBLIC QFLAG, NEWEXEC, RETSAVE, USER_PROC_PDB, HEADSAVE, EXEC_BLOCK
					   PUBLIC COM_LINE, COM_FCB1, COM_FCB2, COM_SSSP, COM_CSIP, NEXTCS
					   PUBLIC NEXTIP, NAMESPEC
				
 0000  41 4C 43 4C 44 4C	REG8	   DB	"ALCLDLBLAHCHDHBH"
       42 4C 41 48 43 48	
       44 48 42 48		
 0010  41 58 43 58 44 58	REG16	   DB	"AXCXDXBXSPBPSIDI"
       42 58 53 50 42 50	
       53 49 44 49		
 0020  45 53 43 53 53 53	SREG	   DB	"ESCSSSDS",0,0
       44 53 00 00		
 002A  42 59 57 4F 44 57	SIZ8	   DB	"BYWODWQWTB",0,0
       51 57 54 42 00 00	
				; 0
 0036  0442 R 0000 E		DISTAB	   DW	OFFSET DG:ADDMN,ALUFROMREG
 003A  0442 R 0000 E			   DW	OFFSET DG:ADDMN,ALUFROMREG
 003E  0442 R 0000 E			   DW	OFFSET DG:ADDMN,ALUTOREG
 0042  0442 R 0000 E			   DW	OFFSET DG:ADDMN,ALUTOREG
 0046  0442 R 0000 E			   DW	OFFSET DG:ADDMN,ACCIMM
 004A  0442 R 0000 E			   DW	OFFSET DG:ADDMN,ACCIMM
 004E  0761 R 0000 E			   DW	OFFSET DG:PUSHMN,SEGOP
 0052  0757 R 0000 E			   DW	OFFSET DG:POPMN,SEGOP
 0056  0456 R 0000 E			   DW	OFFSET DG:ORMN,ALUFROMREG
 005A  0456 R 0000 E			   DW	OFFSET DG:ORMN,ALUFROMREG
 005E  0456 R 0000 E			   DW	OFFSET DG:ORMN,ALUTOREG
 0062  0456 R 0000 E			   DW	OFFSET DG:ORMN,ALUTOREG
 0066  0456 R 0000 E			   DW	OFFSET DG:ORMN,ACCIMM
 006A  0456 R 0000 E			   DW	OFFSET DG:ORMN,ACCIMM
 006E  0761 R 0000 E			   DW	OFFSET DG:PUSHMN,SEGOP
 0072  0757 R 0000 E			   DW	OFFSET DG:POPMN,SEGOP
				; 10H
 0076  0446 R 0000 E			   DW	OFFSET DG:ADCMN,ALUFROMREG
 007A  0446 R 0000 E			   DW	OFFSET DG:ADCMN,ALUFROMREG
 007E  0446 R 0000 E			   DW	OFFSET DG:ADCMN,ALUTOREG
 0082  0446 R 0000 E			   DW	OFFSET DG:ADCMN,ALUTOREG
 0086  0446 R 0000 E			   DW	OFFSET DG:ADCMN,ACCIMM
 008A  0446 R 0000 E			   DW	OFFSET DG:ADCMN,ACCIMM
 008E  0761 R 0000 E			   DW	OFFSET DG:PUSHMN,SEGOP
 0092  0757 R 0000 E			   DW	OFFSET DG:POPMN,SEGOP
 0096  044E R 0000 E			   DW	OFFSET DG:SBBMN,ALUFROMREG
 009A  044E R 0000 E			   DW	OFFSET DG:SBBMN,ALUFROMREG
 009E  044E R 0000 E			   DW	OFFSET DG:SBBMN,ALUTOREG
 00A2  044E R 0000 E			   DW	OFFSET DG:SBBMN,ALUTOREG
 00A6  044E R 0000 E			   DW	OFFSET DG:SBBMN,ACCIMM
 00AA  044E R 0000 E			   DW	OFFSET DG:SBBMN,ACCIMM
 00AE  0761 R 0000 E			   DW	OFFSET DG:PUSHMN,SEGOP
 00B2  0757 R 0000 E			   DW	OFFSET DG:POPMN,SEGOP
				; 20H
 00B6  0459 R 0000 E			   DW	OFFSET DG:ANDMN,ALUFROMREG
 00BA  0459 R 0000 E			   DW	OFFSET DG:ANDMN,ALUFROMREG
 00BE  0459 R 0000 E			   DW	OFFSET DG:ANDMN,ALUTOREG
 00C2  0459 R 0000 E			   DW	OFFSET DG:ANDMN,ALUTOREG
 00C6  0459 R 0000 E			   DW	OFFSET DG:ANDMN,ACCIMM
 00CA  0459 R 0000 E			   DW	OFFSET DG:ANDMN,ACCIMM
 00CE  07E2 R 0000 E			   DW	OFFSET DG:ESSEGMN,ESPRE
 00D2  049A R 0000 E			   DW	OFFSET DG:DAAMN,NOOPERANDS
 00D6  044A R 0000 E			   DW	OFFSET DG:SUBMN,ALUFROMREG
 00DA  044A R 0000 E			   DW	OFFSET DG:SUBMN,ALUFROMREG
 00DE  044A R 0000 E			   DW	OFFSET DG:SUBMN,ALUTOREG
 00E2  044A R 0000 E			   DW	OFFSET DG:SUBMN,ALUTOREG
 00E6  044A R 0000 E			   DW	OFFSET DG:SUBMN,ACCIMM
 00EA  044A R 0000 E			   DW	OFFSET DG:SUBMN,ACCIMM
 00EE  07E6 R 0000 E			   DW	OFFSET DG:CSSEGMN,CSPRE
 00F2  049E R 0000 E			   DW	OFFSET DG:DASMN,NOOPERANDS
				; 30H
 00F6  0452 R 0000 E			   DW	OFFSET DG:XORMN,ALUFROMREG
 00FA  0452 R 0000 E			   DW	OFFSET DG:XORMN,ALUFROMREG
 00FE  0452 R 0000 E			   DW	OFFSET DG:XORMN,ALUTOREG
 0102  0452 R 0000 E			   DW	OFFSET DG:XORMN,ALUTOREG
 0106  0452 R 0000 E			   DW	OFFSET DG:XORMN,ACCIMM
 010A  0452 R 0000 E			   DW	OFFSET DG:XORMN,ACCIMM
 010E  07EA R 0000 E			   DW	OFFSET DG:SSSEGMN,SSPRE
 0112  045D R 0000 E			   DW	OFFSET DG:AAAMN,NOOPERANDS
 0116  0492 R 0000 E			   DW	OFFSET DG:CMPMN,ALUFROMREG
 011A  0492 R 0000 E			   DW	OFFSET DG:CMPMN,ALUFROMREG
Microsoft (R) Macro Assembler Version 5.10                  2/14/25 23:44:19
DEBCONST.ASM                                                Page     1-3
                                                            

 011E  0492 R 0000 E			   DW	OFFSET DG:CMPMN,ALUTOREG
 0122  0492 R 0000 E			   DW	OFFSET DG:CMPMN,ALUTOREG
 0126  0492 R 0000 E			   DW	OFFSET DG:CMPMN,ACCIMM
 012A  0492 R 0000 E			   DW	OFFSET DG:CMPMN,ACCIMM
 012E  07EE R 0000 E			   DW	OFFSET DG:DSSEGMN,DSPRE
 0132  0469 R 0000 E			   DW	OFFSET DG:AASMN,NOOPERANDS
				; 40H
 0136  065D R 0000 E			   DW	OFFSET DG:INCMN,REGOP
 013A  065D R 0000 E			   DW	OFFSET DG:INCMN,REGOP
 013E  065D R 0000 E			   DW	OFFSET DG:INCMN,REGOP
 0142  065D R 0000 E			   DW	OFFSET DG:INCMN,REGOP
 0146  065D R 0000 E			   DW	OFFSET DG:INCMN,REGOP
 014A  065D R 0000 E			   DW	OFFSET DG:INCMN,REGOP
 014E  065D R 0000 E			   DW	OFFSET DG:INCMN,REGOP
 0152  065D R 0000 E			   DW	OFFSET DG:INCMN,REGOP
 0156  04A2 R 0000 E			   DW	OFFSET DG:DECMN,REGOP
 015A  04A2 R 0000 E			   DW	OFFSET DG:DECMN,REGOP
 015E  04A2 R 0000 E			   DW	OFFSET DG:DECMN,REGOP
 0162  04A2 R 0000 E			   DW	OFFSET DG:DECMN,REGOP
 0166  04A2 R 0000 E			   DW	OFFSET DG:DECMN,REGOP
 016A  04A2 R 0000 E			   DW	OFFSET DG:DECMN,REGOP
 016E  04A2 R 0000 E			   DW	OFFSET DG:DECMN,REGOP
 0172  04A2 R 0000 E			   DW	OFFSET DG:DECMN,REGOP
				; 50H
 0176  0761 R 0000 E			   DW	OFFSET DG:PUSHMN,REGOP
 017A  0761 R 0000 E			   DW	OFFSET DG:PUSHMN,REGOP
 017E  0761 R 0000 E			   DW	OFFSET DG:PUSHMN,REGOP
 0182  0761 R 0000 E			   DW	OFFSET DG:PUSHMN,REGOP
 0186  0761 R 0000 E			   DW	OFFSET DG:PUSHMN,REGOP
 018A  0761 R 0000 E			   DW	OFFSET DG:PUSHMN,REGOP
 018E  0761 R 0000 E			   DW	OFFSET DG:PUSHMN,REGOP
 0192  0761 R 0000 E			   DW	OFFSET DG:PUSHMN,REGOP
 0196  0757 R 0000 E			   DW	OFFSET DG:POPMN,REGOP
 019A  0757 R 0000 E			   DW	OFFSET DG:POPMN,REGOP
 019E  0757 R 0000 E			   DW	OFFSET DG:POPMN,REGOP
 01A2  0757 R 0000 E			   DW	OFFSET DG:POPMN,REGOP
 01A6  0757 R 0000 E			   DW	OFFSET DG:POPMN,REGOP
 01AA  0757 R 0000 E			   DW	OFFSET DG:POPMN,REGOP
 01AE  0757 R 0000 E			   DW	OFFSET DG:POPMN,REGOP
 01B2  0757 R 0000 E			   DW	OFFSET DG:POPMN,REGOP
				; 60H
 01B6  0436 R 0000 E			   DW	OFFSET DG:DBMN,SAVHEX
 01BA  0436 R 0000 E			   DW	OFFSET DG:DBMN,SAVHEX
 01BE  0436 R 0000 E			   DW	OFFSET DG:DBMN,SAVHEX
 01C2  0436 R 0000 E			   DW	OFFSET DG:DBMN,SAVHEX
 01C6  0436 R 0000 E			   DW	OFFSET DG:DBMN,SAVHEX
 01CA  0436 R 0000 E			   DW	OFFSET DG:DBMN,SAVHEX
 01CE  0436 R 0000 E			   DW	OFFSET DG:DBMN,SAVHEX
 01D2  0436 R 0000 E			   DW	OFFSET DG:DBMN,SAVHEX
 01D6  0436 R 0000 E			   DW	OFFSET DG:DBMN,SAVHEX
 01DA  0436 R 0000 E			   DW	OFFSET DG:DBMN,SAVHEX
 01DE  0436 R 0000 E			   DW	OFFSET DG:DBMN,SAVHEX
 01E2  0436 R 0000 E			   DW	OFFSET DG:DBMN,SAVHEX
 01E6  0436 R 0000 E			   DW	OFFSET DG:DBMN,SAVHEX
 01EA  0436 R 0000 E			   DW	OFFSET DG:DBMN,SAVHEX
 01EE  0436 R 0000 E			   DW	OFFSET DG:DBMN,SAVHEX
 01F2  0436 R 0000 E			   DW	OFFSET DG:DBMN,SAVHEX
				; 70H
 01F6  06E4 R 0000 E			   DW	OFFSET DG:JOMN,SHORTJMP
 01FA  06E0 R 0000 E			   DW	OFFSET DG:JNOMN,SHORTJMP
 01FE  068B R 0000 E			   DW	OFFSET DG:JCMN,SHORTJMP
 0202  0683 R 0000 E			   DW	OFFSET DG:JNCMN,SHORTJMP
 0206  069E R 0000 E			   DW	OFFSET DG:JZMN,SHORTJMP
 020A  06C8 R 0000 E			   DW	OFFSET DG:JNZMN,SHORTJMP
 020E  0687 R 0000 E			   DW	OFFSET DG:JBEMN,SHORTJMP
 0212  067B R 0000 E			   DW	OFFSET DG:JAMN,SHORTJMP
 0216  06E7 R 0000 E			   DW	OFFSET DG:JSMN,SHORTJMP
 021A  06DC R 0000 E			   DW	OFFSET DG:JNSMN,SHORTJMP
 021E  06D0 R 0000 E			   DW	OFFSET DG:JPEMN,SHORTJMP
 0222  06D4 R 0000 E			   DW	OFFSET DG:JPOMN,SHORTJMP
 0226  06B8 R 0000 E			   DW	OFFSET DG:JLMN,SHORTJMP
 022A  06A4 R 0000 E			   DW	OFFSET DG:JGEMN,SHORTJMP
 022E  06B4 R 0000 E			   DW	OFFSET DG:JLEMN,SHORTJMP
 0232  06A8 R 0000 E			   DW	OFFSET DG:JGMN,SHORTJMP
				; 80H
 0236  0000 0000 E			   DW	0,IMMED
Microsoft (R) Macro Assembler Version 5.10                  2/14/25 23:44:19
DEBCONST.ASM                                                Page     1-4
                                                            

 023A  0000 0000 E			   DW	0,IMMED
 023E  0000 0000 E			   DW	0,IMMED
 0242  0000 0000 E			   DW	0,SIGNIMM
 0246  07CE R 0000 E			   DW	OFFSET DG:TESTMN,ALUTOREG ;ARR 2.4
 024A  07CE R 0000 E			   DW	OFFSET DG:TESTMN,ALUTOREG ;ARR 2.4
 024E  07D8 R 0000 E			   DW	OFFSET DG:XCHGMN,ALUTOREG ;ARR 2.4
 0252  07D8 R 0000 E			   DW	OFFSET DG:XCHGMN,ALUTOREG ;ARR 2.4
 0256  073A R 0000 E			   DW	OFFSET DG:MOVMN,ALUFROMREG
 025A  073A R 0000 E			   DW	OFFSET DG:MOVMN,ALUFROMREG
 025E  073A R 0000 E			   DW	OFFSET DG:MOVMN,ALUTOREG
 0262  073A R 0000 E			   DW	OFFSET DG:MOVMN,ALUTOREG
 0266  073A R 0000 E			   DW	OFFSET DG:MOVMN,MOVSEGTO
 026A  06F6 R 0000 E			   DW	OFFSET DG:LEAMN,WORDTOALU
 026E  073A R 0000 E			   DW	OFFSET DG:MOVMN,MOVSEGFROM
 0272  0757 R 0000 E			   DW	OFFSET DG:POPMN,GETADDR
				; 90H
 0276  0746 R 0000 E			   DW	OFFSET DG:NOPMN,NOOPERANDS
 027A  07D8 R 0000 E			   DW	OFFSET DG:XCHGMN,XCHGAX
 027E  07D8 R 0000 E			   DW	OFFSET DG:XCHGMN,XCHGAX
 0282  07D8 R 0000 E			   DW	OFFSET DG:XCHGMN,XCHGAX
 0286  07D8 R 0000 E			   DW	OFFSET DG:XCHGMN,XCHGAX
 028A  07D8 R 0000 E			   DW	OFFSET DG:XCHGMN,XCHGAX
 028E  07D8 R 0000 E			   DW	OFFSET DG:XCHGMN,XCHGAX
 0292  07D8 R 0000 E			   DW	OFFSET DG:XCHGMN,XCHGAX
 0296  0472 R 0000 E			   DW	OFFSET DG:CBWMN,NOOPERANDS
 029A  0496 R 0000 E			   DW	OFFSET DG:CWDMN,NOOPERANDS
 029E  046D R 0000 E			   DW	OFFSET DG:CALLMN,LONGJMP
 02A2  07D3 R 0000 E			   DW	OFFSET DG:WAITMN,NOOPERANDS
 02A6  075B R 0000 E			   DW	OFFSET DG:PUSHFMN,NOOPERANDS
 02AA  0752 R 0000 E			   DW	OFFSET DG:POPFMN,NOOPERANDS
 02AE  0799 R 0000 E			   DW	OFFSET DG:SAHFMN,NOOPERANDS
 02B2  06ED R 0000 E			   DW	OFFSET DG:LAHFMN,NOOPERANDS
				; A0H
 02B6  073A R 0000 E			   DW	OFFSET DG:MOVMN,LOADACC
 02BA  073A R 0000 E			   DW	OFFSET DG:MOVMN,LOADACC
 02BE  073A R 0000 E			   DW	OFFSET DG:MOVMN,STOREACC
 02C2  073A R 0000 E			   DW	OFFSET DG:MOVMN,STOREACC
 02C6  072E R 0000 E			   DW	OFFSET DG:MOVBMN,NOOPERANDS
 02CA  0734 R 0000 E			   DW	OFFSET DG:MOVWMN,NOOPERANDS
 02CE  0486 R 0000 E			   DW	OFFSET DG:CMPBMN,NOOPERANDS
 02D2  048C R 0000 E			   DW	OFFSET DG:CMPWMN,NOOPERANDS
 02D6  07CE R 0000 E			   DW	OFFSET DG:TESTMN,ACCIMM
 02DA  07CE R 0000 E			   DW	OFFSET DG:TESTMN,ACCIMM
 02DE  07C2 R 0000 E			   DW	OFFSET DG:STOBMN,NOOPERANDS
 02E2  07C8 R 0000 E			   DW	OFFSET DG:STOWMN,NOOPERANDS
 02E6  0703 R 0000 E			   DW	OFFSET DG:LODBMN,NOOPERANDS
 02EA  0709 R 0000 E			   DW	OFFSET DG:LODWMN,NOOPERANDS
 02EE  07A2 R 0000 E			   DW	OFFSET DG:SCABMN,NOOPERANDS
 02F2  07A8 R 0000 E			   DW	OFFSET DG:SCAWMN,NOOPERANDS
				; B0H
 02F6  073A R 0000 E			   DW	OFFSET DG:MOVMN,REGIMMB
 02FA  073A R 0000 E			   DW	OFFSET DG:MOVMN,REGIMMB
 02FE  073A R 0000 E			   DW	OFFSET DG:MOVMN,REGIMMB
 0302  073A R 0000 E			   DW	OFFSET DG:MOVMN,REGIMMB
 0306  073A R 0000 E			   DW	OFFSET DG:MOVMN,REGIMMB
 030A  073A R 0000 E			   DW	OFFSET DG:MOVMN,REGIMMB
 030E  073A R 0000 E			   DW	OFFSET DG:MOVMN,REGIMMB
 0312  073A R 0000 E			   DW	OFFSET DG:MOVMN,REGIMMB
 0316  073A R 0000 E			   DW	OFFSET DG:MOVMN,REGIMMW
 031A  073A R 0000 E			   DW	OFFSET DG:MOVMN,REGIMMW
 031E  073A R 0000 E			   DW	OFFSET DG:MOVMN,REGIMMW
 0322  073A R 0000 E			   DW	OFFSET DG:MOVMN,REGIMMW
 0326  073A R 0000 E			   DW	OFFSET DG:MOVMN,REGIMMW
 032A  073A R 0000 E			   DW	OFFSET DG:MOVMN,REGIMMW
 032E  073A R 0000 E			   DW	OFFSET DG:MOVMN,REGIMMW
 0332  073A R 0000 E			   DW	OFFSET DG:MOVMN,REGIMMW
				; C0H
 0336  0436 R 0000 E			   DW	OFFSET DG:DBMN,SAVHEX
 033A  0436 R 0000 E			   DW	OFFSET DG:DBMN,SAVHEX
 033E  078D R 0000 E			   DW	OFFSET DG:RETMN,SAV16
 0342  078D R 0000 E			   DW	OFFSET DG:RETMN,NOOPERANDS
 0346  06FA R 0000 E			   DW	OFFSET DG:LESMN,WORDTOALU
 034A  06F2 R 0000 E			   DW	OFFSET DG:LDSMN,WORDTOALU
 034E  073A R 0000 E			   DW	OFFSET DG:MOVMN,MEMIMM
 0352  073A R 0000 E			   DW	OFFSET DG:MOVMN,MEMIMM
 0356  0436 R 0000 E			   DW	OFFSET DG:DBMN,SAVHEX
Microsoft (R) Macro Assembler Version 5.10                  2/14/25 23:44:19
DEBCONST.ASM                                                Page     1-5
                                                            

 035A  0436 R 0000 E			   DW	OFFSET DG:DBMN,SAVHEX
 035E  0788 R 0000 E			   DW	OFFSET DG:RETFMN,SAV16
 0362  0788 R 0000 E			   DW	OFFSET DG:RETFMN,NOOPERANDS
 0366  0666 R 0000 E			   DW	OFFSET DG:INTMN,INT3
 036A  0666 R 0000 E			   DW	OFFSET DG:INTMN,SAV8
 036E  0661 R 0000 E			   DW	OFFSET DG:INTOMN,NOOPERANDS
 0372  066D R 0000 E			   DW	OFFSET DG:IRETMN,NOOPERANDS
				; D0H
 0376  0000 0000 E			   DW	0,SHIFT
 037A  0000 0000 E			   DW	0,SHIFT
 037E  0000 0000 E			   DW	0,SHIFTV
 0382  0000 0000 E			   DW	0,SHIFTV
 0386  0465 R 0000 E			   DW	OFFSET DG:AAMMN,CHK10
 038A  0461 R 0000 E			   DW	OFFSET DG:AADMN,CHK10
 038E  0436 R 0000 E			   DW	OFFSET DG:DBMN,SAVHEX
 0392  07DD R 0000 E			   DW	OFFSET DG:XLATMN,NOOPERANDS
 0396  0000 0000 E			   DW	0,M8087 		; d8
 039A  0000 0000 E			   DW	0,M8087_D9		; d9
 039E  0000 0000 E			   DW	0,M8087 		; da
 03A2  0000 0000 E			   DW	0,M8087_DB		; db
 03A6  0000 0000 E			   DW	0,M8087 		; dc
 03AA  0000 0000 E			   DW	0,M8087_DD		; dd
 03AE  0000 0000 E			   DW	0,M8087 		; de
 03B2  0000 0000 E			   DW	0,M8087_DF		; df
				; E0H
 03B6  070F R 0000 E			   DW	OFFSET DG:LOOPNZMN,SHORTJMP
 03BA  0716 R 0000 E			   DW	OFFSET DG:LOOPZMN,SHORTJMP
 03BE  0729 R 0000 E			   DW	OFFSET DG:LOOPMN,SHORTJMP
 03C2  067E R 0000 E			   DW	OFFSET DG:JCXZMN,SHORTJMP
 03C6  066A R 0000 E			   DW	OFFSET DG:INMN,INFIXB
 03CA  066A R 0000 E			   DW	OFFSET DG:INMN,INFIXW
 03CE  074E R 0000 E			   DW	OFFSET DG:OUTMN,OUTFIXB
 03D2  074E R 0000 E			   DW	OFFSET DG:OUTMN,OUTFIXW
 03D6  046D R 0000 E			   DW	OFFSET DG:CALLMN,JMPCALL
 03DA  06C4 R 0000 E			   DW	OFFSET DG:JMPMN,JMPCALL
 03DE  06C4 R 0000 E			   DW	OFFSET DG:JMPMN,LONGJMP
 03E2  06C4 R 0000 E			   DW	OFFSET DG:JMPMN,SHORTJMP
 03E6  066A R 0000 E			   DW	OFFSET DG:INMN,INVARB
 03EA  066A R 0000 E			   DW	OFFSET DG:INMN,INVARW
 03EE  074E R 0000 E			   DW	OFFSET DG:OUTMN,OUTVARB
 03F2  074E R 0000 E			   DW	OFFSET DG:OUTMN,OUTVARW
				; F0H
 03F6  06FE R 0000 E			   DW	OFFSET DG:LOCKMN,PREFIX
 03FA  0436 R 0000 E			   DW	OFFSET DG:DBMN,SAVHEX
 03FE  0773 R 0000 E			   DW	OFFSET DG:REPNZMN,PREFIX
 0402  076E R 0000 E			   DW	OFFSET DG:REPZMN,PREFIX
 0406  064F R 0000 E			   DW	OFFSET DG:HLTMN,NOOPERANDS
 040A  0482 R 0000 E			   DW	OFFSET DG:CMCMN,NOOPERANDS
 040E  0000 0000 E			   DW	0,GRP1
 0412  0000 0000 E			   DW	0,GRP1
 0416  0476 R 0000 E			   DW	OFFSET DG:CLCMN,NOOPERANDS
 041A  07B6 R 0000 E			   DW	OFFSET DG:STCMN,NOOPERANDS
 041E  047E R 0000 E			   DW	OFFSET DG:DIMN,NOOPERANDS
 0422  07BE R 0000 E			   DW	OFFSET DG:EIMN,NOOPERANDS
 0426  047A R 0000 E			   DW	OFFSET DG:UPMN,NOOPERANDS
 042A  07BA R 0000 E			   DW	OFFSET DG:DOWNMN,NOOPERANDS
 042E  0000 0000 E			   DW	0,GRP2
 0432  0000 0000 E			   DW	0,GRP2
				
 0436  44 42 00			DBMN	   DB	"DB",0
 0439  44 57 00				   DB	"DW",0
 043C  3B 00				   DB	";",0
 043E  4F 52 47 00		ORGMN	   DB	"ORG",0
 0442  41 44 44 00		ADDMN	   DB	"ADD",0
 0446  41 44 43 00		ADCMN	   DB	"ADC",0
 044A  53 55 42 00		SUBMN	   DB	"SUB",0
 044E  53 42 42 00		SBBMN	   DB	"SBB",0
 0452  58 4F 52 00		XORMN	   DB	"XOR",0
 0456  4F 52 00			ORMN	   DB	"OR",0
 0459  41 4E 44 00		ANDMN	   DB	"AND",0
 045D  41 41 41 00		AAAMN	   DB	"AAA",0
 0461  41 41 44 00		AADMN	   DB	"AAD",0
 0465  41 41 4D 00		AAMMN	   DB	"AAM",0
 0469  41 41 53 00		AASMN	   DB	"AAS",0
 046D  43 41 4C 4C 00		CALLMN	   DB	"CALL",0
 0472  43 42 57 00		CBWMN	   DB	"CBW",0
Microsoft (R) Macro Assembler Version 5.10                  2/14/25 23:44:19
DEBCONST.ASM                                                Page     1-6
                                                            

 0476  43 4C 43 00		CLCMN	   DB	"CLC",0
 047A  43 4C 44 00		UPMN	   DB	"CLD",0                 ; CLD,0
 047E  43 4C 49 00		DIMN	   DB	"CLI",0
 0482  43 4D 43 00		CMCMN	   DB	"CMC",0
 0486  43 4D 50 53 42 00	CMPBMN	   DB	"CMPSB",0               ; CMPSB
 048C  43 4D 50 53 57 00	CMPWMN	   DB	"CMPSW",0               ; CMPSW,0
 0492  43 4D 50 00		CMPMN	   DB	"CMP",0
 0496  43 57 44 00		CWDMN	   DB	"CWD",0
 049A  44 41 41 00		DAAMN	   DB	"DAA",0
 049E  44 41 53 00		DASMN	   DB	"DAS",0
 04A2  44 45 43 00		DECMN	   DB	"DEC",0
 04A6  44 49 56 00		DIVMN	   DB	"DIV",0
 04AA  45 53 43 00		ESCMN	   DB	"ESC",0
 04AE  46 58 43 48 00			   DB	"FXCH",0
 04B3  46 46 52 45 45 00		   DB	"FFREE",0
 04B9  46 43 4F 4D 50 50		   DB	"FCOMPP",0
       00			
 04C0  46 43 4F 4D 50 00		   DB	"FCOMP",0
 04C6  46 43 4F 4D 00			   DB	"FCOM",0
 04CB  46 49 43 4F 4D 50		   DB	"FICOMP",0
       00			
 04D2  46 49 43 4F 4D 00		   DB	"FICOM",0
 04D8  46 4E 4F 50 00			   DB	"FNOP",0
 04DD  46 43 48 53 00			   DB	"FCHS",0
 04E2  46 41 42 53 00			   DB	"FABS",0
 04E7  46 54 53 54 00			   DB	"FTST",0
 04EC  46 58 41 4D 00			   DB	"FXAM",0
 04F1  46 4C 44 4C 32 54		   DB	"FLDL2T",0
       00			
 04F8  46 4C 44 4C 32 45		   DB	"FLDL2E",0
       00			
 04FF  46 4C 44 4C 47 32		   DB	"FLDLG2",0
       00			
 0506  46 4C 44 4C 4E 32		   DB	"FLDLN2",0
       00			
 050D  46 4C 44 50 49 00		   DB	"FLDPI",0
 0513  46 4C 44 31 00			   DB	"FLD1",0
 0518  46 4C 44 5A 00			   DB	"FLDZ",0
 051D  46 32 58 4D 31 00		   DB	"F2XM1",0
 0523  46 59 4C 32 58 50		   DB	"FYL2XP1",0
       31 00			
 052B  46 59 4C 32 58 00		   DB	"FYL2X",0
 0531  46 50 54 41 4E 00		   DB	"FPTAN",0
 0537  46 50 41 54 41 4E		   DB	"FPATAN",0
       00			
 053E  46 58 54 52 41 43		   DB	"FXTRACT",0
       54 00			
 0546  46 44 45 43 53 54		   DB	"FDECSTP",0
       50 00			
 054E  46 49 4E 43 53 54		   DB	"FINCSTP",0
       50 00			
 0556  46 50 52 45 4D 00		   DB	"FPREM",0
 055C  46 53 51 52 54 00		   DB	"FSQRT",0
 0562  46 52 4E 44 49 4E		   DB	"FRNDINT",0
       54 00			
 056A  46 53 43 41 4C 45		   DB	"FSCALE",0
       00			
 0571  46 49 4E 49 54 00		   DB	"FINIT",0
 0577  46 44 49 53 49 00		   DB	"FDISI",0
 057D  46 45 4E 49 00			   DB	"FENI",0
 0582  46 43 4C 45 58 00		   DB	"FCLEX",0
 0588  46 42 4C 44 00			   DB	"FBLD",0
 058D  46 42 53 54 50 00		   DB	"FBSTP",0
 0593  46 4C 44 43 57 00		   DB	"FLDCW",0
 0599  46 53 54 43 57 00		   DB	"FSTCW",0
 059F  46 53 54 53 57 00		   DB	"FSTSW",0
 05A5  46 53 54 45 4E 56		   DB	"FSTENV",0
       00			
 05AC  46 4C 44 45 4E 56		   DB	"FLDENV",0
       00			
 05B3  46 53 41 56 45 00		   DB	"FSAVE",0
 05B9  46 52 53 54 4F 52		   DB	"FRSTOR",0
       00			
 05C0  46 41 44 44 50 00		   DB	"FADDP",0
 05C6  46 41 44 44 00			   DB	"FADD",0
 05CB  46 49 41 44 44 00		   DB	"FIADD",0
Microsoft (R) Macro Assembler Version 5.10                  2/14/25 23:44:19
DEBCONST.ASM                                                Page     1-7
                                                            

 05D1  46 53 55 42 52 50		   DB	"FSUBRP",0
       00			
 05D8  46 53 55 42 52 00		   DB	"FSUBR",0
 05DE  46 53 55 42 50 00		   DB	"FSUBP",0
 05E4  46 53 55 42 00			   DB	"FSUB",0
 05E9  46 49 53 55 42 52		   DB	"FISUBR",0
       00			
 05F0  46 49 53 55 42 00		   DB	"FISUB",0
 05F6  46 4D 55 4C 50 00		   DB	"FMULP",0
 05FC  46 4D 55 4C 00			   DB	"FMUL",0
 0601  46 49 4D 55 4C 00		   DB	"FIMUL",0
 0607  46 44 49 56 52 50		   DB	"FDIVRP",0
       00			
 060E  46 44 49 56 52 00		   DB	"FDIVR",0
 0614  46 44 49 56 50 00		   DB	"FDIVP",0
 061A  46 44 49 56 00			   DB	"FDIV",0
 061F  46 49 44 49 56 52		   DB	"FIDIVR",0
       00			
 0626  46 49 44 49 56 00		   DB	"FIDIV",0
 062C  46 57 41 49 54 00		   DB	"FWAIT",0
 0632  46 49 4C 44 00			   DB	"FILD",0
 0637  46 4C 44 00			   DB	"FLD",0
 063B  46 53 54 50 00			   DB	"FSTP",0
 0640  46 53 54 00			   DB	"FST",0
 0644  46 49 53 54 50 00		   DB	"FISTP",0
 064A  46 49 53 54 00			   DB	"FIST",0
 064F  48 4C 54 00		HLTMN	   DB	"HLT",0
 0653  49 44 49 56 00		IDIVMN	   DB	"IDIV",0
 0658  49 4D 55 4C 00		IMULMN	   DB	"IMUL",0
 065D  49 4E 43 00		INCMN	   DB	"INC",0
 0661  49 4E 54 4F 00		INTOMN	   DB	"INTO",0
 0666  49 4E 54 00		INTMN	   DB	"INT",0
 066A  49 4E 00			INMN	   DB	"IN",0                  ; IN
 066D  49 52 45 54 00		IRETMN	   DB	"IRET",0
 0672  4A 4E 42 45 00			   DB	"JNBE",0
 0677  4A 41 45 00			   DB	"JAE",0
 067B  4A 41 00			JAMN	   DB	"JA",0
 067E  4A 43 58 5A 00		JCXZMN	   DB	"JCXZ",0
 0683  4A 4E 42 00		JNCMN	   DB	"JNB",0
 0687  4A 42 45 00		JBEMN	   DB	"JBE",0
 068B  4A 42 00			JCMN	   DB	"JB",0
 068E  4A 4E 43 00			   DB	"JNC",0
 0692  4A 43 00				   DB	"JC",0
 0695  4A 4E 41 45 00			   DB	"JNAE",0
 069A  4A 4E 41 00			   DB	"JNA",0
 069E  4A 5A 00			JZMN	   DB	"JZ",0
 06A1  4A 45 00				   DB	"JE",0
 06A4  4A 47 45 00		JGEMN	   DB	"JGE",0
 06A8  4A 47 00			JGMN	   DB	"JG",0
 06AB  4A 4E 4C 45 00			   DB	"JNLE",0
 06B0  4A 4E 4C 00			   DB	"JNL",0
 06B4  4A 4C 45 00		JLEMN	   DB	"JLE",0
 06B8  4A 4C 00			JLMN	   DB	"JL",0
 06BB  4A 4E 47 45 00			   DB	"JNGE",0
 06C0  4A 4E 47 00			   DB	"JNG",0
 06C4  4A 4D 50 00		JMPMN	   DB	"JMP",0
 06C8  4A 4E 5A 00		JNZMN	   DB	"JNZ",0
 06CC  4A 4E 45 00			   DB	"JNE",0
 06D0  4A 50 45 00		JPEMN	   DB	"JPE",0
 06D4  4A 50 4F 00		JPOMN	   DB	"JPO",0
 06D8  4A 4E 50 00			   DB	"JNP",0
 06DC  4A 4E 53 00		JNSMN	   DB	"JNS",0
 06E0  4A 4E 4F 00		JNOMN	   DB	"JNO",0
 06E4  4A 4F 00			JOMN	   DB	"JO",0
 06E7  4A 53 00			JSMN	   DB	"JS",0
 06EA  4A 50 00				   DB	"JP",0
 06ED  4C 41 48 46 00		LAHFMN	   DB	"LAHF",0
 06F2  4C 44 53 00		LDSMN	   DB	"LDS",0
 06F6  4C 45 41 00		LEAMN	   DB	"LEA",0
 06FA  4C 45 53 00		LESMN	   DB	"LES",0
 06FE  4C 4F 43 4B 00		LOCKMN	   DB	"LOCK",0
 0703  4C 4F 44 53 42 00	LODBMN	   DB	"LODSB",0               ; LODSB
 0709  4C 4F 44 53 57 00	LODWMN	   DB	"LODSW",0               ; LODSW,0
 070F  4C 4F 4F 50 4E 5A	LOOPNZMN   DB	"LOOPNZ",0
       00			
 0716  4C 4F 4F 50 5A 00	LOOPZMN    DB	"LOOPZ",0
Microsoft (R) Macro Assembler Version 5.10                  2/14/25 23:44:19
DEBCONST.ASM                                                Page     1-8
                                                            

 071C  4C 4F 4F 50 4E 45		   DB	"LOOPNE",0
       00			
 0723  4C 4F 4F 50 45 00		   DB	"LOOPE",0
 0729  4C 4F 4F 50 00		LOOPMN	   DB	"LOOP",0
 072E  4D 4F 56 53 42 00	MOVBMN	   DB	"MOVSB",0               ; MOVSB
 0734  4D 4F 56 53 57 00	MOVWMN	   DB	"MOVSW",0               ; MOVSW,0
 073A  4D 4F 56 00		MOVMN	   DB	"MOV",0
 073E  4D 55 4C 00		MULMN	   DB	"MUL",0
 0742  4E 45 47 00		NEGMN	   DB	"NEG",0
 0746  4E 4F 50 00		NOPMN	   DB	"NOP",0
 074A  4E 4F 54 00		NOTMN	   DB	"NOT",0
 074E  4F 55 54 00		OUTMN	   DB	"OUT",0                 ; OUT
 0752  50 4F 50 46 00		POPFMN	   DB	"POPF",0
 0757  50 4F 50 00		POPMN	   DB	"POP",0
 075B  50 55 53 48 46 00	PUSHFMN    DB	"PUSHF",0
 0761  50 55 53 48 00		PUSHMN	   DB	"PUSH",0
 0766  52 43 4C 00		RCLMN	   DB	"RCL",0
 076A  52 43 52 00		RCRMN	   DB	"RCR",0
 076E  52 45 50 5A 00		REPZMN	   DB	"REPZ",0
 0773  52 45 50 4E 5A 00	REPNZMN    DB	"REPNZ",0
 0779  52 45 50 45 00			   DB	"REPE",0
 077E  52 45 50 4E 45 00		   DB	"REPNE",0
 0784  52 45 50 00			   DB	"REP",0
 0788  52 45 54 46 00		RETFMN	   DB	"RETF",0
 078D  52 45 54 00		RETMN	   DB	"RET",0
 0791  52 4F 4C 00		ROLMN	   DB	"ROL",0
 0795  52 4F 52 00		RORMN	   DB	"ROR",0
 0799  53 41 48 46 00		SAHFMN	   DB	"SAHF",0
 079E  53 41 52 00		SARMN	   DB	"SAR",0
 07A2  53 43 41 53 42 00	SCABMN	   DB	"SCASB",0               ; SCASB
 07A8  53 43 41 53 57 00	SCAWMN	   DB	"SCASW",0               ; SCASW,0
 07AE  53 48 4C 00		SHLMN	   DB	"SHL",0
 07B2  53 48 52 00		SHRMN	   DB	"SHR",0
 07B6  53 54 43 00		STCMN	   DB	"STC",0
 07BA  53 54 44 00		DOWNMN	   DB	"STD",0                 ; STD
 07BE  53 54 49 00		EIMN	   DB	"STI",0                 ; STI
 07C2  53 54 4F 53 42 00	STOBMN	   DB	"STOSB",0               ; STOSB
 07C8  53 54 4F 53 57 00	STOWMN	   DB	"STOSW",0               ; STOSW,0
 07CE  54 45 53 54 00		TESTMN	   DB	"TEST",0
 07D3  57 41 49 54 00		WAITMN	   DB	"WAIT",0
 07D8  58 43 48 47 00		XCHGMN	   DB	"XCHG",0
 07DD  58 4C 41 54 00		XLATMN	   DB	"XLAT",0
 07E2  45 53 3A 00		ESSEGMN    DB	"ES:",0
 07E6  43 53 3A 00		CSSEGMN    DB	"CS:",0
 07EA  53 53 3A 00		SSSEGMN    DB	"SS:",0
 07EE  44 53 3A 00		DSSEGMN    DB	"DS:",0
 07F2  3F 3F 3F 00		BADMN	   DB	"???",0
				
 07F6  41 44 44 24 4D 55	M8087_TAB  DB	"ADD$MUL$COM$COMP$SUB$SUBR$DIV$DIVR$"
       4C 24 43 4F 4D 24	
       43 4F 4D 50 24 53	
       55 42 24 53 55 42	
       52 24 44 49 56 24	
       44 49 56 52 24		
 0819  46 24 46 49 24 46	FI_TAB	   DB	"F$FI$F$FI$"
       24 46 49 24		
 0823  44 57 4F 52 44 20	SIZE_TAB   DB	"DWORD PTR $DWORD PTR $QWORD PTR $WORD PTR $"
       50 54 52 20 24 44	
       57 4F 52 44 20 50	
       54 52 20 24 51 57	
       4F 52 44 20 50 54	
       52 20 24 57 4F 52	
       44 20 50 54 52 20	
       24			
 084E  42 59 54 45 20 50		   DB	"BYTE PTR $TBYTE PTR $"
       54 52 20 24 54 42	
       59 54 45 20 50 54	
       52 20 24			
				
 0863  4C 44 24 40 24 53	MD9_TAB    DB	"LD$@$ST$STP$LDENV$LDCW$STENV$STCW$"
       54 24 53 54 50 24	
       4C 44 45 4E 56 24	
       4C 44 43 57 24 53	
       54 45 4E 56 24 53	
       54 43 57 24		
 0885  43 48 53 24 41 42	MD9_TAB2   DB	"CHS$ABS$@$@$TST$XAM$@$@$LD1$LDL2T$LDL2E$"
Microsoft (R) Macro Assembler Version 5.10                  2/14/25 23:44:19
DEBCONST.ASM                                                Page     1-9
                                                            

       53 24 40 24 40 24	
       54 53 54 24 58 41	
       4D 24 40 24 40 24	
       4C 44 31 24 4C 44	
       4C 32 54 24 4C 44	
       4C 32 45 24		
 08AD  4C 44 50 49 24 4C		   DB	"LDPI$LDLG2$LDLN2$LDZ$@$2XM1$YL2X$PTAN$PATAN$XTRACT$"
       44 4C 47 32 24 4C	
       44 4C 4E 32 24 4C	
       44 5A 24 40 24 32	
       58 4D 31 24 59 4C	
       32 58 24 50 54 41	
       4E 24 50 41 54 41	
       4E 24 58 54 52 41	
       43 54 24			
 08E0  40 24 44 45 43 53		   DB	"@$DECSTP$INCSTP$PREM$YL2XP1$SQRT$@$RNDINT$SCALE$@$@$"
       54 50 24 49 4E 43	
       53 54 50 24 50 52	
       45 4D 24 59 4C 32	
       58 50 31 24 53 51	
       52 54 24 40 24 52	
       4E 44 49 4E 54 24	
       53 43 41 4C 45 24	
       40 24 40 24		
				
 0914  49 4C 44 24 40 24	MDB_TAB    DB	"ILD$@$IST$ISTP$@$LD$@$STP$"
       49 53 54 24 49 53	
       54 50 24 40 24 4C	
       44 24 40 24 53 54	
       50 24			
 092E  45 4E 49 24 44 49	MDB_TAB2   DB	"ENI$DISI$CLEX$INIT$"
       53 49 24 43 4C 45	
       58 24 49 4E 49 54	
       24			
				
 0941  4C 44 24 40 24 53	MDD_TAB    DB	"LD$@$ST$STP$RSTOR$@$SAVE$STSW$"
       54 24 53 54 50 24	
       52 53 54 4F 52 24	
       40 24 53 41 56 45	
       24 53 54 53 57 24	
 095F  46 52 45 45 24 58	MDD_TAB2   DB	"FREE$XCH$ST$STP$"
       43 48 24 53 54 24	
       53 54 50 24		
				
 096F  49 4C 44 24 40 24	MDF_TAB    DB	"ILD$@$IST$ISTP$BLD$ILD$BSTP$ISTP$"
       49 53 54 24 49 53	
       54 50 24 42 4C 44	
       24 49 4C 44 24 42	
       53 54 50 24 49 53	
       54 50 24			
				
				
 0990  FF			OPTAB	   DB	11111111B		; DB
 0991  0000 E				   DW	DB_OPER
 0993  FF				   DB	11111111B		; DW
 0994  0000 E				   DW	DW_OPER
 0996  FF				   DB	11111111B		; COMMENT
 0997  0000 E				   DW	ASSEMLOOP
 0999  FF				   DB	11111111B		; ORG
 099A  0000 E				   DW	DOORG
 099C  00				   DB	0 * 8			; ADD
 099D  0000 E				   DW	GROUP2
 099F  10				   DB	2 * 8			; ADC
 09A0  0000 E				   DW	GROUP2
 09A2  28				   DB	5 * 8			; SUB
 09A3  0000 E				   DW	GROUP2
 09A5  18				   DB	3 * 8			; SBB
 09A6  0000 E				   DW	GROUP2
 09A8  30				   DB	6 * 8			; XOR
 09A9  0000 E				   DW	GROUP2
 09AB  08				   DB	1 * 8			; OR
 09AC  0000 E				   DW	GROUP2
 09AE  20				   DB	4 * 8			; AND
 09AF  0000 E				   DW	GROUP2
 09B1  37				   DB	00110111B		; AAA
 09B2  0000 E				   DW	NO_OPER
Microsoft (R) Macro Assembler Version 5.10                  2/14/25 23:44:19
DEBCONST.ASM                                                Page     1-10
                                                            

 09B4  D5				   DB	11010101B		; AAD
 09B5  0000 E				   DW	AA_OPER
 09B7  D4				   DB	11010100B		; AAM
 09B8  0000 E				   DW	AA_OPER
 09BA  3F				   DB	00111111B		; AAS
 09BB  0000 E				   DW	NO_OPER
 09BD  10				   DB	2 * 8			; CALL
 09BE  0000 E				   DW	CALL_OPER
 09C0  98				   DB	10011000B		; CBW
 09C1  0000 E				   DW	NO_OPER
 09C3  F8				   DB	11111000B		; CLC
 09C4  0000 E				   DW	NO_OPER
 09C6  FC				   DB	11111100B		; CLD
 09C7  0000 E				   DW	NO_OPER
 09C9  FA				   DB	11111010B		; DIM
 09CA  0000 E				   DW	NO_OPER
 09CC  F5				   DB	11110101B		; CMC
 09CD  0000 E				   DW	NO_OPER
 09CF  A6				   DB	10100110B		; CMPB
 09D0  0000 E				   DW	NO_OPER
 09D2  A7				   DB	10100111B		; CMPW
 09D3  0000 E				   DW	NO_OPER
 09D5  38				   DB	7 * 8			; CMP
 09D6  0000 E				   DW	GROUP2
 09D8  99				   DB	10011001B		; CWD
 09D9  0000 E				   DW	NO_OPER
 09DB  27				   DB	00100111B		; DAA
 09DC  0000 E				   DW	NO_OPER
 09DE  2F				   DB	00101111B		; DAS
 09DF  0000 E				   DW	NO_OPER
 09E1  08				   DB	1 * 8			; DEC
 09E2  0000 E				   DW	DCINC_OPER
 09E4  30				   DB	6 * 8			; DIV
 09E5  0000 E				   DW	GROUP1
 09E7  D8				   DB	11011000B		; ESC
 09E8  0000 E				   DW	ESC_OPER
 09EA  09				   DB	00001001B		; FXCH
 09EB  0000 E				   DW	FGROUPP
 09ED  28				   DB	00101000B		; FFREE
 09EE  0000 E				   DW	FGROUPP
 09F0  D9				   DB	11011001B		; FCOMPP
 09F1  0000 E				   DW	FDE_OPER
 09F3  03				   DB	00000011B		; FCOMP
 09F4  0000 E				   DW	FGROUPX 		; Exception to normal P instructions
 09F6  02				   DB	00000010B		; FCOM
 09F7  0000 E				   DW	FGROUPX
 09F9  13				   DB	00010011B		; FICOMP
 09FA  0000 E				   DW	FGROUPZ
 09FC  12				   DB	00010010B		; FICOM
 09FD  0000 E				   DW	FGROUPZ
 09FF  D0				   DB	11010000B		; FNOP
 0A00  0000 E				   DW	FD9_OPER
 0A02  E0				   DB	11100000B		; FCHS
 0A03  0000 E				   DW	FD9_OPER
 0A05  E1				   DB	11100001B		; FABS
 0A06  0000 E				   DW	FD9_OPER
 0A08  E4				   DB	11100100B		; FTST
 0A09  0000 E				   DW	FD9_OPER
 0A0B  E5				   DB	11100101B		; FXAM
 0A0C  0000 E				   DW	FD9_OPER
 0A0E  E9				   DB	11101001B		; FLDL2T
 0A0F  0000 E				   DW	FD9_OPER
 0A11  EA				   DB	11101010B		; FLDL2E
 0A12  0000 E				   DW	FD9_OPER
 0A14  EC				   DB	11101100B		; FLDLG2
 0A15  0000 E				   DW	FD9_OPER
 0A17  ED				   DB	11101101B		; FLDLN2
 0A18  0000 E				   DW	FD9_OPER
 0A1A  EB				   DB	11101011B		; FLDPI
 0A1B  0000 E				   DW	FD9_OPER
 0A1D  E8				   DB	11101000B		; FLD1
 0A1E  0000 E				   DW	FD9_OPER
 0A20  EE				   DB	11101110B		; FLDZ
 0A21  0000 E				   DW	FD9_OPER
 0A23  F0				   DB	11110000B		; F2XM1
 0A24  0000 E				   DW	FD9_OPER
Microsoft (R) Macro Assembler Version 5.10                  2/14/25 23:44:19
DEBCONST.ASM                                                Page     1-11
                                                            

 0A26  F9				   DB	11111001B		; FYL2XP1
 0A27  0000 E				   DW	FD9_OPER
 0A29  F1				   DB	11110001B		; FYL2X
 0A2A  0000 E				   DW	FD9_OPER
 0A2C  F2				   DB	11110010B		; FPTAN
 0A2D  0000 E				   DW	FD9_OPER
 0A2F  F3				   DB	11110011B		; FPATAN
 0A30  0000 E				   DW	FD9_OPER
 0A32  F4				   DB	11110100B		; FXTRACT
 0A33  0000 E				   DW	FD9_OPER
 0A35  F6				   DB	11110110B		; FDECSTP
 0A36  0000 E				   DW	FD9_OPER
 0A38  F7				   DB	11110111B		; FINCSTP
 0A39  0000 E				   DW	FD9_OPER
 0A3B  F8				   DB	11111000B		; FPREM
 0A3C  0000 E				   DW	FD9_OPER
 0A3E  FA				   DB	11111010B		; FSQRT
 0A3F  0000 E				   DW	FD9_OPER
 0A41  FC				   DB	11111100B		; FRNDINT
 0A42  0000 E				   DW	FD9_OPER
 0A44  FD				   DB	11111101B		; FSCALE
 0A45  0000 E				   DW	FD9_OPER
 0A47  E3				   DB	11100011B		; FINIT
 0A48  0000 E				   DW	FDB_OPER
 0A4A  E1				   DB	11100001B		; FDISI
 0A4B  0000 E				   DW	FDB_OPER
 0A4D  E0				   DB	11100000B		; FENI
 0A4E  0000 E				   DW	FDB_OPER
 0A50  E2				   DB	11100010B		; FCLEX
 0A51  0000 E				   DW	FDB_OPER
 0A53  3C				   DB	00111100B		; FBLD
 0A54  0000 E				   DW	FGROUPB
 0A56  3E				   DB	00111110B		; FBSTP
 0A57  0000 E				   DW	FGROUPB
 0A59  0D				   DB	00001101B		; FLDCW
 0A5A  0000 E				   DW	FGROUP3W
 0A5C  0F				   DB	00001111B		; FSTCW
 0A5D  0000 E				   DW	FGROUP3W
 0A5F  2F				   DB	00101111B		; FSTSW
 0A60  0000 E				   DW	FGROUP3W
 0A62  0E				   DB	00001110B		; FSTENV
 0A63  0000 E				   DW	FGROUP3
 0A65  0C				   DB	00001100B		; FLDENV
 0A66  0000 E				   DW	FGROUP3
 0A68  2E				   DB	00101110B		; FSAVE
 0A69  0000 E				   DW	FGROUP3
 0A6B  2C				   DB	00101100B		; FRSTOR
 0A6C  0000 E				   DW	FGROUP3
 0A6E  30				   DB	00110000B		; FADDP
 0A6F  0000 E				   DW	FGROUPP
 0A71  00				   DB	00000000B		; FADD
 0A72  0000 E				   DW	FGROUP
 0A74  10				   DB	00010000B		; FIADD
 0A75  0000 E				   DW	FGROUPZ
 0A77  34				   DB	00110100B		; FSUBRP
 0A78  0000 E				   DW	FGROUPP
 0A7A  05				   DB	00000101B		; FSUBR
 0A7B  0000 E				   DW	FGROUPDS
 0A7D  35				   DB	00110101B		; FSUBP
 0A7E  0000 E				   DW	FGROUPP
 0A80  04				   DB	00000100B		; FSUB
 0A81  0000 E				   DW	FGROUPDS
 0A83  15				   DB	00010101B		; FISUBR
 0A84  0000 E				   DW	FGROUPZ
 0A86  14				   DB	00010100B		; FISUB
 0A87  0000 E				   DW	FGROUPZ
 0A89  31				   DB	00110001B		; FMULP
 0A8A  0000 E				   DW	FGROUPP
 0A8C  01				   DB	00000001B		; FMUL
 0A8D  0000 E				   DW	FGROUP
 0A8F  11				   DB	00010001B		; FIMUL
 0A90  0000 E				   DW	FGROUPZ
 0A92  36				   DB	00110110B		; FDIVRP
 0A93  0000 E				   DW	FGROUPP
 0A95  07				   DB	00000111B		; FDIVR
 0A96  0000 E				   DW	FGROUPDS
Microsoft (R) Macro Assembler Version 5.10                  2/14/25 23:44:19
DEBCONST.ASM                                                Page     1-12
                                                            

 0A98  37				   DB	00110111B		; FDIVP
 0A99  0000 E				   DW	FGROUPP
 0A9B  06				   DB	00000110B		; FDIV
 0A9C  0000 E				   DW	FGROUPDS
 0A9E  17				   DB	00010111B		; FIDIVR
 0A9F  0000 E				   DW	FGROUPZ
 0AA1  16				   DB	00010110B		; FIDIV
 0AA2  0000 E				   DW	FGROUPZ
 0AA4  9B				   DB	10011011B		; FWAIT
 0AA5  0000 E				   DW	NO_OPER
 0AA7  18				   DB	00011000B		; FILD
 0AA8  0000 E				   DW	FGROUPZ
 0AAA  08				   DB	00001000B		; FLD
 0AAB  0000 E				   DW	FGROUPX
 0AAD  0B				   DB	00001011B		; FSTP
 0AAE  0000 E				   DW	FGROUP			;an000; dms;
 0AB0  2A				   DB	00101010B		; FST
 0AB1  0000 E				   DW	FGROUPX
 0AB3  1B				   DB	00011011B		; FISTP
 0AB4  0000 E				   DW	FGROUPZ
 0AB6  1A				   DB	00011010B		; FIST
 0AB7  0000 E				   DW	FGROUPZ
 0AB9  F4				   DB	11110100B		; HLT
 0ABA  0000 E				   DW	NO_OPER
 0ABC  38				   DB	7 * 8			; IDIV
 0ABD  0000 E				   DW	GROUP1
 0ABF  28				   DB	5 * 8			; IMUL
 0AC0  0000 E				   DW	GROUP1
 0AC2  00				   DB	0 * 8			; INC
 0AC3  0000 E				   DW	DCINC_OPER
 0AC5  CE				   DB	11001110B		; INTO
 0AC6  0000 E				   DW	NO_OPER
 0AC8  CC				   DB	11001100B		; INTM
 0AC9  0000 E				   DW	INT_OPER
 0ACB  EC				   DB	11101100B		; IN
 0ACC  0000 E				   DW	IN_OPER
 0ACE  CF				   DB	11001111B		; IRET
 0ACF  0000 E				   DW	NO_OPER
 0AD1  77				   DB	01110111B		; JNBE
 0AD2  0000 E				   DW	DISP8_OPER
 0AD4  73				   DB	01110011B		; JAE
 0AD5  0000 E				   DW	DISP8_OPER
 0AD7  77				   DB	01110111B		; JA
 0AD8  0000 E				   DW	DISP8_OPER
 0ADA  E3				   DB	11100011B		; JCXZ
 0ADB  0000 E				   DW	DISP8_OPER
 0ADD  73				   DB	01110011B		; JNB
 0ADE  0000 E				   DW	DISP8_OPER
 0AE0  76				   DB	01110110B		; JBE
 0AE1  0000 E				   DW	DISP8_OPER
 0AE3  72				   DB	01110010B		; JB
 0AE4  0000 E				   DW	DISP8_OPER
 0AE6  73				   DB	01110011B		; JNC
 0AE7  0000 E				   DW	DISP8_OPER
 0AE9  72				   DB	01110010B		; JC
 0AEA  0000 E				   DW	DISP8_OPER
 0AEC  72				   DB	01110010B		; JNAE
 0AED  0000 E				   DW	DISP8_OPER
 0AEF  76				   DB	01110110B		; JNA
 0AF0  0000 E				   DW	DISP8_OPER
 0AF2  74				   DB	01110100B		; JZ
 0AF3  0000 E				   DW	DISP8_OPER
 0AF5  74				   DB	01110100B		; JE
 0AF6  0000 E				   DW	DISP8_OPER
 0AF8  7D				   DB	01111101B		; JGE
 0AF9  0000 E				   DW	DISP8_OPER
 0AFB  7F				   DB	01111111B		; JG
 0AFC  0000 E				   DW	DISP8_OPER
 0AFE  7F				   DB	01111111B		; JNLE
 0AFF  0000 E				   DW	DISP8_OPER
 0B01  7D				   DB	01111101B		; JNL
 0B02  0000 E				   DW	DISP8_OPER
 0B04  7E				   DB	01111110B		; JLE
 0B05  0000 E				   DW	DISP8_OPER
 0B07  7C				   DB	01111100B		; JL
 0B08  0000 E				   DW	DISP8_OPER
Microsoft (R) Macro Assembler Version 5.10                  2/14/25 23:44:19
DEBCONST.ASM                                                Page     1-13
                                                            

 0B0A  7C				   DB	01111100B		; JNGE
 0B0B  0000 E				   DW	DISP8_OPER
 0B0D  7E				   DB	01111110B		; JNG
 0B0E  0000 E				   DW	DISP8_OPER
 0B10  20				   DB	4 * 8			; JMP
 0B11  0000 E				   DW	JMP_OPER
 0B13  75				   DB	01110101B		; JNZ
 0B14  0000 E				   DW	DISP8_OPER
 0B16  75				   DB	01110101B		; JNE
 0B17  0000 E				   DW	DISP8_OPER
 0B19  7A				   DB	01111010B		; JPE
 0B1A  0000 E				   DW	DISP8_OPER
 0B1C  7B				   DB	01111011B		; JPO
 0B1D  0000 E				   DW	DISP8_OPER
 0B1F  7B				   DB	01111011B		; JNP
 0B20  0000 E				   DW	DISP8_OPER
 0B22  79				   DB	01111001B		; JNS
 0B23  0000 E				   DW	DISP8_OPER
 0B25  71				   DB	01110001B		; JNO
 0B26  0000 E				   DW	DISP8_OPER
 0B28  70				   DB	01110000B		; JO
 0B29  0000 E				   DW	DISP8_OPER
 0B2B  78				   DB	01111000B		; JS
 0B2C  0000 E				   DW	DISP8_OPER
 0B2E  7A				   DB	01111010B		; JP
 0B2F  0000 E				   DW	DISP8_OPER
 0B31  9F				   DB	10011111B		; LAHF
 0B32  0000 E				   DW	NO_OPER
 0B34  C5				   DB	11000101B		; LDS
 0B35  0000 E				   DW	L_OPER
 0B37  8D				   DB	10001101B		; LEA
 0B38  0000 E				   DW	L_OPER
 0B3A  C4				   DB	11000100B		; LES
 0B3B  0000 E				   DW	L_OPER
 0B3D  F0				   DB	11110000B		; LOCK
 0B3E  0000 E				   DW	NO_OPER
 0B40  AC				   DB	10101100B		; LODB
 0B41  0000 E				   DW	NO_OPER
 0B43  AD				   DB	10101101B		; LODW
 0B44  0000 E				   DW	NO_OPER
 0B46  E0				   DB	11100000B		; LOOPNZ
 0B47  0000 E				   DW	DISP8_OPER
 0B49  E1				   DB	11100001B		; LOOPZ
 0B4A  0000 E				   DW	DISP8_OPER
 0B4C  E0				   DB	11100000B		; LOOPNE
 0B4D  0000 E				   DW	DISP8_OPER
 0B4F  E1				   DB	11100001B		; LOOPE
 0B50  0000 E				   DW	DISP8_OPER
 0B52  E2				   DB	11100010B		; LOOP
 0B53  0000 E				   DW	DISP8_OPER
 0B55  A4				   DB	10100100B		; MOVB
 0B56  0000 E				   DW	NO_OPER
 0B58  A5				   DB	10100101B		; MOVW
 0B59  0000 E				   DW	NO_OPER
 0B5B  C6				   DB	11000110B		; MOV
 0B5C  0000 E				   DW	MOV_OPER
 0B5E  20				   DB	4 * 8			; MUL
 0B5F  0000 E				   DW	GROUP1
 0B61  18				   DB	3 * 8			; NEG
 0B62  0000 E				   DW	GROUP1
 0B64  90				   DB	10010000B		; NOP
 0B65  0000 E				   DW	NO_OPER
 0B67  10				   DB	2 * 8			; NOT
 0B68  0000 E				   DW	GROUP1
 0B6A  EE				   DB	11101110B		; OUT
 0B6B  0000 E				   DW	OUT_OPER
 0B6D  9D				   DB	10011101B		; POPF
 0B6E  0000 E				   DW	NO_OPER
 0B70  00				   DB	0 * 8			; POP
 0B71  0000 E				   DW	POP_OPER
 0B73  9C				   DB	10011100B		; PUSHF
 0B74  0000 E				   DW	NO_OPER
 0B76  30				   DB	6 * 8			; PUSH
 0B77  0000 E				   DW	PUSH_OPER
 0B79  10				   DB	2 * 8			; RCL
 0B7A  0000 E				   DW	ROTOP
Microsoft (R) Macro Assembler Version 5.10                  2/14/25 23:44:19
DEBCONST.ASM                                                Page     1-14
                                                            

 0B7C  18				   DB	3 * 8			; RCR
 0B7D  0000 E				   DW	ROTOP
 0B7F  F3				   DB	11110011B		; REPZ
 0B80  0000 E				   DW	NO_OPER
 0B82  F2				   DB	11110010B		; REPNZ
 0B83  0000 E				   DW	NO_OPER
 0B85  F3				   DB	11110011B		; REPE
 0B86  0000 E				   DW	NO_OPER
 0B88  F2				   DB	11110010B		; REPNE
 0B89  0000 E				   DW	NO_OPER
 0B8B  F3				   DB	11110011B		; REP
 0B8C  0000 E				   DW	NO_OPER
 0B8E  CB				   DB	11001011B		; RETF
 0B8F  0000 E				   DW	GET_DATA16
 0B91  C3				   DB	11000011B		; RET
 0B92  0000 E				   DW	GET_DATA16
 0B94  00				   DB	0 * 8			; ROL
 0B95  0000 E				   DW	ROTOP
 0B97  08				   DB	1 * 8			; ROR
 0B98  0000 E				   DW	ROTOP
 0B9A  9E				   DB	10011110B		; SAHF
 0B9B  0000 E				   DW	NO_OPER
 0B9D  38				   DB	7 * 8			; SAR
 0B9E  0000 E				   DW	ROTOP
 0BA0  AE				   DB	10101110B		; SCAB
 0BA1  0000 E				   DW	NO_OPER
 0BA3  AF				   DB	10101111B		; SCAW
 0BA4  0000 E				   DW	NO_OPER
 0BA6  20				   DB	4 * 8			; SHL
 0BA7  0000 E				   DW	ROTOP
 0BA9  28				   DB	5 * 8			; SHR
 0BAA  0000 E				   DW	ROTOP
 0BAC  F9				   DB	11111001B		; STC
 0BAD  0000 E				   DW	NO_OPER
 0BAF  FD				   DB	11111101B		; STD
 0BB0  0000 E				   DW	NO_OPER
 0BB2  FB				   DB	11111011B		; EI
 0BB3  0000 E				   DW	NO_OPER
 0BB5  AA				   DB	10101010B		; STOB
 0BB6  0000 E				   DW	NO_OPER
 0BB8  AB				   DB	10101011B		; STOW
 0BB9  0000 E				   DW	NO_OPER
 0BBB  F6				   DB	11110110B		; TEST
 0BBC  0000 E				   DW	TST_OPER
 0BBE  9B				   DB	10011011B		; WAIT
 0BBF  0000 E				   DW	NO_OPER
 0BC1  86				   DB	10000110B		; XCHG
 0BC2  0000 E				   DW	EX_OPER
 0BC4  D7				   DB	11010111B		; XLAT
 0BC5  0000 E				   DW	NO_OPER
 0BC7  26				   DB	00100110B		; ESSEG
 0BC8  0000 E				   DW	NO_OPER
 0BCA  2E				   DB	00101110B		; CSSEG
 0BCB  0000 E				   DW	NO_OPER
 0BCD  36				   DB	00110110B		; SSSEG
 0BCE  0000 E				   DW	NO_OPER
 0BD0  3E				   DB	00111110B		; DSSEG
 0BD1  0000 E				   DW	NO_OPER
				
 0BD3				ZZOPCODE   LABEL BYTE
 = 00C1				MAXOP	   =	(ZZOPCODE-OPTAB)/3
				
 0BD3  0791 R 0795 R 0766 R	SHFTAB	   DW	OFFSET DG:ROLMN,OFFSET DG:RORMN,OFFSET DG:RCLMN
 0BD9  076A R 07AE R 07B2 R		   DW	OFFSET DG:RCRMN,OFFSET DG:SHLMN,OFFSET DG:SHRMN
 0BDF  07F2 R 079E R			   DW	OFFSET DG:BADMN,OFFSET DG:SARMN
				
 0BE3  0442 R 0456 R 0446 R	IMMTAB	   DW	OFFSET DG:ADDMN,OFFSET DG:ORMN,OFFSET DG:ADCMN
 0BE9  044E R 0459 R 044A R		   DW	OFFSET DG:SBBMN,OFFSET DG:ANDMN,OFFSET DG:SUBMN
 0BEF  0452 R 0492 R			   DW	OFFSET DG:XORMN,OFFSET DG:CMPMN
				
 0BF3  07CE R 07F2 R 074A R	GRP1TAB    DW	OFFSET DG:TESTMN,OFFSET DG:BADMN,OFFSET DG:NOTMN
 0BF9  0742 R 073E R 0658 R		   DW	OFFSET DG:NEGMN,OFFSET DG:MULMN,OFFSET DG:IMULMN
 0BFF  04A6 R 0653 R			   DW	OFFSET DG:DIVMN,OFFSET DG:IDIVMN
				
 0C03  065D R 04A2 R 046D R	GRP2TAB    DW	OFFSET DG:INCMN,OFFSET DG:DECMN,OFFSET DG:CALLMN
 0C09  046D R 06C4 R 06C4 R		   DW	OFFSET DG:CALLMN,OFFSET DG:JMPMN,OFFSET DG:JMPMN
Microsoft (R) Macro Assembler Version 5.10                  2/14/25 23:44:19
DEBCONST.ASM                                                Page     1-15
                                                            

 0C0F  0761 R 07F2 R			   DW	OFFSET DG:PUSHMN,OFFSET DG:BADMN
				
 0C13  0D97 R 0D9B R 0D99 R	SEGTAB	   DW	OFFSET DG:ESSAVE,OFFSET DG:CSSAVE,OFFSET DG:SSSAVE
 0C19  0D95 R				   DW	OFFSET DG:DSSAVE
				
 0C1B  41 58 00 42 58 00	REGTAB	   DB	"AX",0,"BX",0,"CX",0,"DX",0,"SP",0,"BP",0
       43 58 00 44 58 00	
       53 50 00 42 50 00	
 0C2D  53 49 00 44 49 00		   DB	"SI",0,"DI",0,"DS",0,"ES",0,"SS",0,"CS",0,"IP",0,"PC",0
       44 53 00 45 53 00	
       53 53 00 43 53 00	
       49 50 00 50 43 00	
 0C45				REGTABEND  LABEL WORD
				
				; Flags are ordered to correspond with the bits of the flag
				; register, most significant bit first, zero if bit is not
				; a flag. First 16 entries are for bit set, second 16 for
				; bit reset.
				
 0C45  0000			FLAGTAB    DW	0
 0C47  0000				   DW	0
 0C49  0000				   DW	0
 0C4B  0000				   DW	0
 0C4D  4F 56				   DB	"OV"
 0C4F  44 4E				   DB	"DN"
 0C51  45 49				   DB	"EI"                    ; "STI"
 0C53  0000				   DW	0
 0C55  4E 47				   DB	"NG"
 0C57  5A 52				   DB	"ZR"
 0C59  0000				   DW	0
 0C5B  41 43				   DB	"AC"
 0C5D  0000				   DW	0
 0C5F  50 45				   DB	"PE"
 0C61  0000				   DW	0
 0C63  43 59				   DB	"CY"
 0C65  0000				   DW	0
 0C67  0000				   DW	0
 0C69  0000				   DW	0
 0C6B  0000				   DW	0
 0C6D  4E 56				   DB	"NV"
 0C6F  55 50				   DB	"UP"                    ; "CLD"
 0C71  44 49				   DB	"DI"
 0C73  0000				   DW	0
 0C75  50 4C				   DB	"PL"
 0C77  4E 5A				   DB	"NZ"
 0C79  0000				   DW	0
 0C7B  4E 41				   DB	"NA"
 0C7D  0000				   DW	0
 0C7F  50 4F				   DB	"PO"
 0C81  0000				   DW	0
 0C83  4E 43				   DB	"NC"
				
 0C85  0080[				   DW	80H DUP(?)
	   ????			
			 ]	
				
 0D85				STACK	   LABEL BYTE
				
				
				; Register save area
				
 0D85  0000			AXSAVE	   DW	0
 0D87  0000			BXSAVE	   DW	0
 0D89  0000			CXSAVE	   DW	0
 0D8B  0000			DXSAVE	   DW	0
 0D8D  005A			SPSAVE	   DW	5AH
 0D8F  0000			BPSAVE	   DW	0
 0D91  0000			SISAVE	   DW	0
 0D93  0000			DISAVE	   DW	0
 0D95  0000			DSSAVE	   DW	0
 0D97  0000			ESSAVE	   DW	0
 0D99				RSTACK	   LABEL WORD			; Stack set here so registers can be saved by pushing
 0D99  0000			SSSAVE	   DW	0
 0D9B  0000			CSSAVE	   DW	0
 0D9D  0100			IPSAVE	   DW	100H
 0D9F  F202			FLSAVE	    DW	 0F202H
Microsoft (R) Macro Assembler Version 5.10                  2/14/25 23:44:19
DEBCONST.ASM                                                Page     1-16
                                                            

				
 0DA1  00			RSETFLAG   DB	0
				
 = 016A				REGDIF	   EQU	AXSAVE-REGTAB
				
				; This value is initially 0, it is set to non-zero if a file is specified
				;  either at debug invokation, or via the (N)ame command. It is used to
				;  control the printing of the NONAMESPEC message for the (W)rite command.
 0DA2  00			NAMESPEC   DB	0
				
				; RAM area.
				
 0DA3  3F			RDFLG	   DB	READ
 0DA4  0D			TOTREG	   DB	13
 0DA5  0F			DSIZ	   DB	0FH			;changed to 7 if screen 40 col mode
 0DA6  08			NOREGL	   DB	8			;changed to 4 if screen 40 col mode
 0DA7  0080			DISPB	   DW	128			;changed to 64 if screen 40 col mode
				
 0DA9  50			LBUFSIZ    DB	BUFLEN
 0DAA  00			LBUFFCNT   DB	0
 0DAB  0D			LINEBUF    DB	0DH
 0DAC  0050[				   DB	BUFLEN DUP (?)
	   ??			
			 ]	
				
 0DFC  00			PFLAG	   DB	0
 0DFD  00			COLPOS	   DB	0
				
				
 0DFE  00			QFLAG	   DB	0
 0DFF  00			NEWEXEC    DB	0
 0E00  0000			RETSAVE    DW	?
				
 0E02  0000			USER_PROC_PDB DW ?
 0E04  0000			NextCS	   DW	?
 0E06  0000			NextIP	   DW	?
				
 0E08  0000			HEADSAVE   DW	?
				
 0E0A				EXEC_BLOCK LABEL BYTE
 0E0A  0000				   DW	0
 0E0C				COM_LINE   LABEL DWORD
 0E0C  0080				   DW	80H
 0E0E  0000				   DW	?
 0E10				COM_FCB1   LABEL DWORD
 0E10  005C				   DW	FCB
 0E12  0000				   DW	?
 0E14				COM_FCB2   LABEL DWORD
 0E14  006C				   DW	FCB + 10H
 0E16  0000				   DW	?
 0E18  00000000			COM_SSSP   DD	?
 0E1C  00000000			COM_CSIP   DD	?
				
 0E20				CONST	   ENDS
					   END

Microsoft (R) Macro Assembler Version 5.10                  2/14/25 23:44:19
DEBCONST.ASM                                                Symbols-1


Macros:

		N a m e			Lines

ARGVAR . . . . . . . . . . . . .  	  23
ASMVAR . . . . . . . . . . . . .  	   3
ASMVARS  . . . . . . . . . . . .  	   3
ASSERT . . . . . . . . . . . . .  	   0
CALLINSTALL  . . . . . . . . . .  	  12
DOSASSUME  . . . . . . . . . . .  	   3
ENTER  . . . . . . . . . . . . .  	   3
ENTERCRIT  . . . . . . . . . . .  	   1
ERRNZ  . . . . . . . . . . . . .  	   4
FMT  . . . . . . . . . . . . . .  	   0
LEAVE  . . . . . . . . . . . . .  	   2
LEAVECRIT  . . . . . . . . . . .  	   1
LOCALVAR . . . . . . . . . . . .  	  23

Structures and Records:

                N a m e                 Width   # fields
                                        Shift   Width   Mask    Initial

ARENA  . . . . . . . . . . . . .  	0010	0005
  ARENA_SIGNATURE  . . . . . . .  	0000
  ARENA_OWNER  . . . . . . . . .  	0001
  ARENA_SIZE . . . . . . . . . .  	0003
  ARENA_RESERVED . . . . . . . .  	0005
  ARENA_NAME . . . . . . . . . .  	0008
A_BPB  . . . . . . . . . . . . .  	001F	000F
  BPB_BYTESPERSECTOR . . . . . .  	0000
  BPB_SECTORSPERCLUSTER  . . . .  	0002
  BPB_RESERVEDSECTORS  . . . . .  	0003
  BPB_NUMBEROFFATS . . . . . . .  	0005
  BPB_ROOTENTRIES  . . . . . . .  	0006
  BPB_TOTALSECTORS . . . . . . .  	0008
  BPB_MEDIADESCRIPTOR  . . . . .  	000A
  BPB_SECTORSPERFAT  . . . . . .  	000B
  BPB_SECTORSPERTRACK  . . . . .  	000D
  BPB_HEADS  . . . . . . . . . .  	000F
  BPB_HIDDENSECTORS  . . . . . .  	0011
  BPB_BIGTOTALSECTORS  . . . . .  	0015
BPBLOCK  . . . . . . . . . . . .  	000D	0008
  BPSECSZ  . . . . . . . . . . .  	0000
  BPCLUS . . . . . . . . . . . .  	0002
  BPRES  . . . . . . . . . . . .  	0003
  BPFTCNT  . . . . . . . . . . .  	0005
  BPDRCNT  . . . . . . . . . . .  	0006
  BPSCCNT  . . . . . . . . . . .  	0008
  BPMEDIA  . . . . . . . . . . .  	000A
  BPFTSEC  . . . . . . . . . . .  	000B
BUFFER_HASH_ENTRY  . . . . . . .  	0008	0004
  EMS_PAGE_NUM . . . . . . . . .  	0000
  BUFFER_BUCKET  . . . . . . . .  	0002
  DIRTY_COUNT  . . . . . . . . .  	0006
  BUFFER_RESERVED  . . . . . . .  	0007
BUFFINFO . . . . . . . . . . . .  	0023	000F
  HASH_PTR . . . . . . . . . . .  	0000
  HASH_COUNT . . . . . . . . . .  	0004
  CACHE_PTR  . . . . . . . . . .  	0006
  CACHE_COUNT  . . . . . . . . .  	000A
  EMS_SAFE_FLAG  . . . . . . . .  	000C
  EMS_LAST_PAGE  . . . . . . . .  	000D
  EMS_FIRST_PAGE . . . . . . . .  	0011
  EMS_NPA640 . . . . . . . . . .  	0015
  EMS_MODE . . . . . . . . . . .  	0017
  EMS_HANDLE . . . . . . . . . .  	0018
  EMS_PAGEFRAME_NUMBER . . . . .  	001A
  EMS_SEG_CNT  . . . . . . . . .  	001C
  EMS_PAGE_FRAME . . . . . . . .  	001E
  EMS_RESERVED . . . . . . . . .  	0020
  EMS_MAP_BUFF . . . . . . . . .  	0022
CURDIR_LIST  . . . . . . . . . .  	0058	000A
  CURDIR_TEXT  . . . . . . . . .  	0000
  CURDIR_FLAGS . . . . . . . . .  	0043
  CURDIR_DEVPTR  . . . . . . . .  	0045
Microsoft (R) Macro Assembler Version 5.10                  2/14/25 23:44:19
DEBCONST.ASM                                                Symbols-2


  CURDIR_ID  . . . . . . . . . .  	0049
  CURDIR_USER_WORD . . . . . . .  	004D
  CURDIR_END . . . . . . . . . .  	004F
  CURDIR_TYPE  . . . . . . . . .  	0051
  CURDIR_IFS_HDR . . . . . . . .  	0052
  CURDIR_FSDA  . . . . . . . . .  	0056
DIR_ENTRY  . . . . . . . . . . .  	0020	000B
  DIR_NAME . . . . . . . . . . .  	0000
  DIR_ATTR . . . . . . . . . . .  	000B
  DIR_CODEPG . . . . . . . . . .  	000C
  DIR_EXTCLUSTER . . . . . . . .  	000E
  DIR_ATTR2  . . . . . . . . . .  	0010
  DIR_PAD  . . . . . . . . . . .  	0011
  DIR_TIME . . . . . . . . . . .  	0016
  DIR_DATE . . . . . . . . . . .  	0018
  DIR_FIRST  . . . . . . . . . .  	001A
  DIR_SIZE_L . . . . . . . . . .  	001C
  DIR_SIZE_H . . . . . . . . . .  	001E
DPB  . . . . . . . . . . . . . .  	0021	0012
  DPB_DRIVE  . . . . . . . . . .  	0000
  DPB_UNIT . . . . . . . . . . .  	0001
  DPB_SECTOR_SIZE  . . . . . . .  	0002
  DPB_CLUSTER_MASK . . . . . . .  	0004
  DPB_CLUSTER_SHIFT  . . . . . .  	0005
  DPB_FIRST_FAT  . . . . . . . .  	0006
  DPB_FAT_COUNT  . . . . . . . .  	0008
  DPB_ROOT_ENTRIES . . . . . . .  	0009
  DPB_FIRST_SECTOR . . . . . . .  	000B
  DPB_MAX_CLUSTER  . . . . . . .  	000D
  DPB_FAT_SIZE . . . . . . . . .  	000F
  DPB_DIR_SECTOR . . . . . . . .  	0011
  DPB_DRIVER_ADDR  . . . . . . .  	0013
  DPB_MEDIA  . . . . . . . . . .  	0017
  DPB_FIRST_ACCESS . . . . . . .  	0018
  DPB_NEXT_DPB . . . . . . . . .  	0019
  DPB_NEXT_FREE  . . . . . . . .  	001D
  DPB_FREE_CNT . . . . . . . . .  	001F
EXEC0  . . . . . . . . . . . . .  	000E	0004
  EXEC0_ENVIRON  . . . . . . . .  	0000
  EXEC0_COM_LINE . . . . . . . .  	0002
  EXEC0_5C_FCB . . . . . . . . .  	0006
  EXEC0_6C_FCB . . . . . . . . .  	000A
EXEC1  . . . . . . . . . . . . .  	0016	0008
  EXEC1_ENVIRON  . . . . . . . .  	0000
  EXEC1_COM_LINE . . . . . . . .  	0002
  EXEC1_5C_FCB . . . . . . . . .  	0006
  EXEC1_6C_FCB . . . . . . . . .  	000A
  EXEC1_SP . . . . . . . . . . .  	000E
  EXEC1_SS . . . . . . . . . . .  	0010
  EXEC1_IP . . . . . . . . . . .  	0012
  EXEC1_CS . . . . . . . . . . .  	0014
EXEC3  . . . . . . . . . . . . .  	0004	0002
  EXEC3_LOAD_ADDR  . . . . . . .  	0000
  EXEC3_RELOC_FAC  . . . . . . .  	0002
EXE_FILE . . . . . . . . . . . .  	0020	000F
  EXE_SIGNATURE  . . . . . . . .  	0000
  EXE_LEN_MOD_512  . . . . . . .  	0002
  EXE_PAGES  . . . . . . . . . .  	0004
  EXE_RLE_COUNT  . . . . . . . .  	0006
  EXE_PAR_DIR  . . . . . . . . .  	0008
  EXE_MIN_BSS  . . . . . . . . .  	000A
  EXE_MAX_BSS  . . . . . . . . .  	000C
  EXE_SS . . . . . . . . . . . .  	000E
  EXE_SP . . . . . . . . . . . .  	0010
  EXE_CHKSUM . . . . . . . . . .  	0012
  EXE_IP . . . . . . . . . . . .  	0014
  EXE_CS . . . . . . . . . . . .  	0016
  EXE_RLE_TABLE  . . . . . . . .  	0018
  EXE_IOV  . . . . . . . . . . .  	001A
  EXE_SYM_TAB  . . . . . . . . .  	001C
EXT_OPEN_PARM  . . . . . . . . .  	0006	0002
  EXT_SET_LIST . . . . . . . . .  	0000
  EXT_NUM_OF_PARM  . . . . . . .  	0004
FIND_BUF . . . . . . . . . . . .  	002B	000C
  FIND_BUF_DRIVE . . . . . . . .  	0000
  FIND_BUF_NAME  . . . . . . . .  	0001
Microsoft (R) Macro Assembler Version 5.10                  2/14/25 23:44:19
DEBCONST.ASM                                                Symbols-3


  FIND_BUF_SATTR . . . . . . . .  	000C
  FIND_BUF_LASTENT . . . . . . .  	000D
  FIND_BUF_DIRSTART  . . . . . .  	000F
  FIND_BUF_NETID . . . . . . . .  	0011
  FIND_BUF_ATTR  . . . . . . . .  	0015
  FIND_BUF_TIME  . . . . . . . .  	0016
  FIND_BUF_DATE  . . . . . . . .  	0018
  FIND_BUF_SIZE_L  . . . . . . .  	001A
  FIND_BUF_SIZE_H  . . . . . . .  	001C
  FIND_BUF_PNAME . . . . . . . .  	001E
INTERNAT_BLOCK . . . . . . . . .  	0018	0015
  DATE_TIM_FORMAT  . . . . . . .  	0000
  CURRENCY_SYM . . . . . . . . .  	0002
  THOUS_SEP  . . . . . . . . . .  	0007
  DECIMAL_SEP  . . . . . . . . .  	0009
  DATE_SEP . . . . . . . . . . .  	000B
  TIME_SEP . . . . . . . . . . .  	000D
  BIT_FIELD  . . . . . . . . . .  	000F
  CURRENCY_CENTS . . . . . . . .  	0010
  TIME_24  . . . . . . . . . . .  	0011
  MAP_CALL . . . . . . . . . . .  	0012
  DATA_SEP . . . . . . . . . . .  	0016
PROCESS_DATA_BLOCK . . . . . . .  	005C	0011
  PDB_EXIT_CALL  . . . . . . . .  	0000
  PDB_BLOCK_LEN  . . . . . . . .  	0002
  PDB_CPM_CALL . . . . . . . . .  	0005
  PDB_EXIT . . . . . . . . . . .  	000A
  PDB_CTRL_C . . . . . . . . . .  	000E
  PDB_FATAL_ABORT  . . . . . . .  	0012
  PDB_PARENT_PID . . . . . . . .  	0016
  PDB_JFN_TABLE  . . . . . . . .  	0018
  PDB_ENVIRON  . . . . . . . . .  	002C
  PDB_USER_STACK . . . . . . . .  	002E
  PDB_JFN_LENGTH . . . . . . . .  	0032
  PDB_JFN_POINTER  . . . . . . .  	0034
  PDB_NEXT_PDB . . . . . . . . .  	0038
  PDB_PAD1 . . . . . . . . . . .  	003C
  PDB_CALL_SYSTEM  . . . . . . .  	0050
  PDB_PAD2 . . . . . . . . . . .  	0055
SF . . . . . . . . . . . . . . .  	0008	0003
  SFLINK . . . . . . . . . . . .  	0000
  SFCOUNT  . . . . . . . . . . .  	0004
  SFTABLE  . . . . . . . . . . .  	0006
SF_ENTRY . . . . . . . . . . . .  	003B	0014
  SF_REF_COUNT . . . . . . . . .  	0000
  SF_MODE  . . . . . . . . . . .  	0002
  SF_ATTR  . . . . . . . . . . .  	0004
  SF_FLAGS . . . . . . . . . . .  	0005
  SF_DEVPTR  . . . . . . . . . .  	0007
  SF_FIRCLUS . . . . . . . . . .  	000B
  SF_TIME  . . . . . . . . . . .  	000D
  SF_DATE  . . . . . . . . . . .  	000F
  SF_SIZE  . . . . . . . . . . .  	0011
  SF_POSITION  . . . . . . . . .  	0015
  SF_CLUSPOS . . . . . . . . . .  	0019
  SF_DIRSEC  . . . . . . . . . .  	001B
  SF_DIRPOS  . . . . . . . . . .  	001F
  SF_NAME  . . . . . . . . . . .  	0020
  SF_CHAIN . . . . . . . . . . .  	002B
  SF_UID . . . . . . . . . . . .  	002F
  SF_PID . . . . . . . . . . . .  	0031
  SF_MFT . . . . . . . . . . . .  	0033
  SF_LSTCLUS . . . . . . . . . .  	0035
  SF_IFS_HDR . . . . . . . . . .  	0037
SYMBOL_ENTRY . . . . . . . . . .  	0106	0004
  SYM_VALUE  . . . . . . . . . .  	0000
  SYM_TYPE . . . . . . . . . . .  	0004
  SYM_LEN  . . . . . . . . . . .  	0006
  SYM_NAME . . . . . . . . . . .  	0007
SYSINITVARS  . . . . . . . . . .  	0047	0018
  SYSI_DPB . . . . . . . . . . .  	0000
  SYSI_SFT . . . . . . . . . . .  	0004
  SYSI_CLOCK . . . . . . . . . .  	0008
  SYSI_CON . . . . . . . . . . .  	000C
  SYSI_MAXSEC  . . . . . . . . .  	0010
  SYSI_BUF . . . . . . . . . . .  	0012
Microsoft (R) Macro Assembler Version 5.10                  2/14/25 23:44:19
DEBCONST.ASM                                                Symbols-4


  SYSI_CDS . . . . . . . . . . .  	0016
  SYSI_FCB . . . . . . . . . . .  	001A
  SYSI_KEEP  . . . . . . . . . .  	001E
  SYSI_NUMIO . . . . . . . . . .  	0020
  SYSI_NCDS  . . . . . . . . . .  	0021
  SYSI_DEV . . . . . . . . . . .  	0022
  SYSI_ATTR  . . . . . . . . . .  	0026
  SYSI_STRAT . . . . . . . . . .  	0028
  SYSI_INTER . . . . . . . . . .  	002A
  SYSI_NAME  . . . . . . . . . .  	002C
  SYSI_SPLICE  . . . . . . . . .  	0034
  SYSI_IBMDOS_SIZE . . . . . . .  	0035
  SYSI_IFS_DOSCALL@  . . . . . .  	0037
  SYSI_IFS . . . . . . . . . . .  	003B
  SYSI_BUFFERS . . . . . . . . .  	003F
  SYSI_BOOT_DRIVE  . . . . . . .  	0043
  SYSI_DWMOVE  . . . . . . . . .  	0044
  SYSI_EXT_MEM . . . . . . . . .  	0045
SYSINITVARS_EXT  . . . . . . . .  	0008	0002
  SYSI_INITVARS  . . . . . . . .  	0000
  SYSI_COUNTRY_TAB . . . . . . .  	0004
SYS_FCB  . . . . . . . . . . . .  	0025	000C
  FCB_DRIVE  . . . . . . . . . .  	0000
  FCB_NAME . . . . . . . . . . .  	0001
  FCB_EXT  . . . . . . . . . . .  	0009
  FCB_EXTENT . . . . . . . . . .  	000C
  FCB_RECSIZ . . . . . . . . . .  	000E
  FCB_FILSIZ . . . . . . . . . .  	0010
  FCB_DRVBP  . . . . . . . . . .  	0012
  FCB_FDATE  . . . . . . . . . .  	0014
  FCB_FTIME  . . . . . . . . . .  	0016
  FCB_RESERVED . . . . . . . . .  	0018
  FCB_NR . . . . . . . . . . . .  	0020
  FCB_RR . . . . . . . . . . . .  	0021
USER_ENVIRON . . . . . . . . . .  	0018	000C
  USER_AX  . . . . . . . . . . .  	0000
  USER_BX  . . . . . . . . . . .  	0002
  USER_CX  . . . . . . . . . . .  	0004
  USER_DX  . . . . . . . . . . .  	0006
  USER_SI  . . . . . . . . . . .  	0008
  USER_DI  . . . . . . . . . . .  	000A
  USER_BP  . . . . . . . . . . .  	000C
  USER_DS  . . . . . . . . . . .  	000E
  USER_ES  . . . . . . . . . . .  	0010
  USER_IP  . . . . . . . . . . .  	0012
  USER_CS  . . . . . . . . . . .  	0014
  USER_F . . . . . . . . . . . .  	0016

Segments and Groups:

                N a m e         	Length	 Align	Combine Class

DG . . . . . . . . . . . . . . .  	GROUP
  CODE . . . . . . . . . . . . .  	0000	BYTE	PUBLIC	
  CONST  . . . . . . . . . . . .  	0E20	BYTE	PUBLIC	
  CSTACK . . . . . . . . . . . .  	0000	PARA	STACK	
  DATA . . . . . . . . . . . . .  	0000	BYTE	PUBLIC	

Symbols:            

                N a m e         	Type	 Value	 Attr

AAAMN  . . . . . . . . . . . . .  	L BYTE	045D	CONST	Global
AADMN  . . . . . . . . . . . . .  	L BYTE	0461	CONST	Global
AAMMN  . . . . . . . . . . . . .  	L BYTE	0465	CONST
AASMN  . . . . . . . . . . . . .  	L BYTE	0469	CONST	Global
AA_OPER  . . . . . . . . . . . .  	L NEAR	0000	CODE	External
ABORT  . . . . . . . . . . . . .  	NUMBER	0000	
ACCESS_MASK  . . . . . . . . . .  	NUMBER	000F	
ACCIMM . . . . . . . . . . . . .  	L NEAR	0000	CODE	External
ACTION_CREATED_OPENED  . . . . .  	NUMBER	0002	
ACTION_OPENED  . . . . . . . . .  	NUMBER	0001	
ACTION_REPLACED_OPENED . . . . .  	NUMBER	0003	
ADCMN  . . . . . . . . . . . . .  	L BYTE	0446	CONST	Global
ADDMN  . . . . . . . . . . . . .  	L BYTE	0442	CONST	Global
Microsoft (R) Macro Assembler Version 5.10                  2/14/25 23:44:19
DEBCONST.ASM                                                Symbols-5


ADDR_INT_ABORT . . . . . . . . .  	NUMBER	0080	
ADDR_INT_COMMAND . . . . . . . .  	NUMBER	0084	
ADDR_INT_CTRL_C  . . . . . . . .  	NUMBER	008C	
ADDR_INT_DISK_READ . . . . . . .  	NUMBER	0094	
ADDR_INT_DISK_WRITE  . . . . . .  	NUMBER	0098	
ADDR_INT_FASTCON . . . . . . . .  	NUMBER	00A4	
ADDR_INT_FATAL_ABORT . . . . . .  	NUMBER	0090	
ADDR_INT_IBM . . . . . . . . . .  	NUMBER	00A8	
ADDR_INT_KEEP_PROCESS  . . . . .  	NUMBER	009C	
ADDR_INT_SPOOLER . . . . . . . .  	NUMBER	00A0	
ADDR_INT_TERMINATE . . . . . . .  	NUMBER	0088	
ALLOC  . . . . . . . . . . . . .  	NUMBER	0048	
ALLOCOPER  . . . . . . . . . . .  	NUMBER	0058	
ALLOWED_FAIL . . . . . . . . . .  	NUMBER	0008	
ALLOWED_IGNORE . . . . . . . . .  	NUMBER	0020	
ALLOWED_RETRY  . . . . . . . . .  	NUMBER	0010	
ALTVECT  . . . . . . . . . . . .  	ALIAS	 FALSE		
ALT_EXPECTED_VERSION . . . . . .  	NUMBER	1A05	
ALT_MAJOR_VERSION  . . . . . . .  	NUMBER	0005	
ALT_MINOR_VERSION  . . . . . . .  	NUMBER	001A	
ALUFROMREG . . . . . . . . . . .  	L NEAR	0000	CODE	External
ALUTOREG . . . . . . . . . . . .  	L NEAR	0000	CODE	External
ANDMN  . . . . . . . . . . . . .  	L BYTE	0459	CONST	Global
ARENA_OWNER_SYSTEM . . . . . . .  	NUMBER	0000	
ARENA_SIGNATURE_END  . . . . . .  	NUMBER	005A	
ARENA_SIGNATURE_NORMAL . . . . .  	NUMBER	004D	
ASSEMLOOP  . . . . . . . . . . .  	L NEAR	0000	CODE	External
ASSIGNOPER . . . . . . . . . . .  	NUMBER	005F	
ATTR_ALL . . . . . . . . . . . .  	NUMBER	0016	
ATTR_ARCHIVE . . . . . . . . . .  	NUMBER	0020	
ATTR_CHANGEABLE  . . . . . . . .  	NUMBER	0027	
ATTR_DEVICE  . . . . . . . . . .  	NUMBER	0040	
ATTR_DIRECTORY . . . . . . . . .  	NUMBER	0010	
ATTR_HIDDEN  . . . . . . . . . .  	NUMBER	0002	
ATTR_IGNORE  . . . . . . . . . .  	NUMBER	0061	
ATTR_READ_ONLY . . . . . . . . .  	NUMBER	0001	
ATTR_SYSTEM  . . . . . . . . . .  	NUMBER	0004	
ATTR_VOLUME_ID . . . . . . . . .  	NUMBER	0008	
AUTO_COMMIT_WRITE  . . . . . . .  	NUMBER	4000	
AXSAVE . . . . . . . . . . . . .  	L WORD	0D85	CONST	Global

BADMN  . . . . . . . . . . . . .  	L BYTE	07F2	CONST	Global
BPLEN  . . . . . . . . . . . . .  	NUMBER	0032	
BPMAX  . . . . . . . . . . . . .  	NUMBER	000A	
BPREG  . . . . . . . . . . . . .  	NUMBER	5042	
BPSAVE . . . . . . . . . . . . .  	L WORD	0D8F	CONST	Global
BUFFERFLAG . . . . . . . . . . .  	NUMBER	FFFF	
BUFINSIZ . . . . . . . . . . . .  	NUMBER	0014	
BUFLEN . . . . . . . . . . . . .  	NUMBER	0050	
BUFSIZ . . . . . . . . . . . . .  	NUMBER	0200	
BUF_DIRTY  . . . . . . . . . . .  	NUMBER	0040	
BUF_DPB  . . . . . . . . . . . .  		000D	
BUF_FILL . . . . . . . . . . . .  		0011	
BUF_FLAGS  . . . . . . . . . . .  		0005	
BUF_FREE . . . . . . . . . . . .  	NUMBER	00FF	
BUF_ID . . . . . . . . . . . . .  		0004	
BUF_ISDATA . . . . . . . . . . .  	NUMBER	0008	
BUF_ISDIR  . . . . . . . . . . .  	NUMBER	0004	
BUF_ISFAT  . . . . . . . . . . .  	NUMBER	0002	
BUF_ISNET  . . . . . . . . . . .  	NUMBER	0080	
BUF_NETID  . . . . . . . . . . .  	ALIAS	 BUFINSIZ		
BUF_NEXT . . . . . . . . . . . .  		0000	
BUF_OFFSET . . . . . . . . . . .  	DWORD	0006	
BUF_PREV . . . . . . . . . . . .  		0002	
BUF_RESERVED . . . . . . . . . .  		0013	
BUF_SECTOR . . . . . . . . . . .  		0006	
BUF_SNBUF  . . . . . . . . . . .  	NUMBER	0010	
BUF_TYPE_0 . . . . . . . . . . .  	NUMBER	00F1	
BUF_VISIT  . . . . . . . . . . .  	NUMBER	0020	
BUF_WRTCNT . . . . . . . . . . .  		000A	
BUF_WRTCNTINC  . . . . . . . . .  		000B	
BXREG  . . . . . . . . . . . . .  	NUMBER	5842	
BXSAVE . . . . . . . . . . . . .  	L WORD	0D87	CONST	Global

CALLMN . . . . . . . . . . . . .  	L BYTE	046D	CONST	Global
CALL_OPER  . . . . . . . . . . .  	L NEAR	0000	CODE	External
Microsoft (R) Macro Assembler Version 5.10                  2/14/25 23:44:19
DEBCONST.ASM                                                Symbols-6


CARGS  . . . . . . . . . . . . .  	NUMBER	0000	
CBWMN  . . . . . . . . . . . . .  	L BYTE	0472	CONST	Global
CHAR_AT_SIGN . . . . . . . . . .  	NUMBER	0040	
CHAR_BACKSPACE . . . . . . . . .  	NUMBER	0008	
CHAR_BLANK . . . . . . . . . . .  	NUMBER	0020	
CHAR_COLON . . . . . . . . . . .  	NUMBER	003A	
CHAR_COMMA . . . . . . . . . . .  	NUMBER	002C	
CHAR_EOF . . . . . . . . . . . .  	NUMBER	001A	
CHAR_EQUAL . . . . . . . . . . .  	NUMBER	003D	
CHAR_LEFT_BRACKET  . . . . . . .  	NUMBER	005B	
CHAR_MINUS . . . . . . . . . . .  	NUMBER	002D	
CHAR_OPER  . . . . . . . . . . .  	NUMBER	0037	
CHAR_PERIOD  . . . . . . . . . .  	NUMBER	002E	
CHAR_RUBOUT  . . . . . . . . . .  	NUMBER	007F	
CHAR_SEMICOLON . . . . . . . . .  	NUMBER	003B	
CHAR_TAB . . . . . . . . . . . .  	NUMBER	0009	
CHAR_ZERO  . . . . . . . . . . .  	NUMBER	0030	
CHDIR  . . . . . . . . . . . . .  	NUMBER	003B	
CHK10  . . . . . . . . . . . . .  	L NEAR	0000	CODE	External
CHMOD  . . . . . . . . . . . . .  	NUMBER	0043	
CLCMN  . . . . . . . . . . . . .  	L BYTE	0476	CONST
CLOSE  . . . . . . . . . . . . .  	NUMBER	003E	
CMCMN  . . . . . . . . . . . . .  	L BYTE	0482	CONST	Global
CMPBMN . . . . . . . . . . . . .  	L BYTE	0486	CONST
CMPMN  . . . . . . . . . . . . .  	L BYTE	0492	CONST	Global
CMPWMN . . . . . . . . . . . . .  	L BYTE	048C	CONST
COLPOS . . . . . . . . . . . . .  	L BYTE	0DFD	CONST	Global
COMMA  . . . . . . . . . . . . .  	NUMBER	2C00	
COMMIT . . . . . . . . . . . . .  	NUMBER	0068	
COM_CSIP . . . . . . . . . . . .  	L DWORD	0E1C	CONST	Global
COM_FCB1 . . . . . . . . . . . .  	L DWORD	0E10	CONST	Global
COM_FCB2 . . . . . . . . . . . .  	L DWORD	0E14	CONST	Global
COM_LINE . . . . . . . . . . . .  	L DWORD	0E0C	CONST	Global
COM_SSSP . . . . . . . . . . . .  	L DWORD	0E18	CONST	Global
CR . . . . . . . . . . . . . . .  	NUMBER	000D	
CREAT  . . . . . . . . . . . . .  	NUMBER	003C	
CREATENEWFILE  . . . . . . . . .  	NUMBER	005B	
CREATETEMPFILE . . . . . . . . .  	NUMBER	005A	
CREATE_PROCESS_DATA_BLOCK  . . .  	NUMBER	0026	
CRITASSIGN . . . . . . . . . . .  	NUMBER	0008	
CRITDEVICE . . . . . . . . . . .  	NUMBER	0002	
CRITDISK . . . . . . . . . . . .  	NUMBER	0001	
CRITIFS  . . . . . . . . . . . .  	NUMBER	0006	
CRITMEM  . . . . . . . . . . . .  	NUMBER	0001	
CRITNET  . . . . . . . . . . . .  	NUMBER	0005	
CRITSFT  . . . . . . . . . . . .  	NUMBER	0001	
CRITSHARE  . . . . . . . . . . .  	NUMBER	0001	
CSPRE  . . . . . . . . . . . . .  	L NEAR	0000	CODE	External
CSSAVE . . . . . . . . . . . . .  	L WORD	0D9B	CONST	Global
CSSEGMN  . . . . . . . . . . . .  	L BYTE	07E6	CONST	Global
CURDIRLEN  . . . . . . . . . . .  	NUMBER	0058	
CURDIR_INUSE . . . . . . . . . .  	NUMBER	4000	
CURDIR_ISIFS . . . . . . . . . .  	NUMBER	8000	
CURDIR_ISNET . . . . . . . . . .  	NUMBER	8000	
CURDIR_LOCAL . . . . . . . . . .  	NUMBER	1000	
CURDIR_NETID . . . . . . . . . .  	DWORD	0049	
CURDIR_SPLICE  . . . . . . . . .  	NUMBER	2000	
CURRENT_DIR  . . . . . . . . . .  	NUMBER	0047	
CWDMN  . . . . . . . . . . . . .  	L BYTE	0496	CONST	Global
CXSAVE . . . . . . . . . . . . .  	L WORD	0D89	CONST	Global
C_BS . . . . . . . . . . . . . .  	NUMBER	0008	
C_CR . . . . . . . . . . . . . .  	NUMBER	000D	
C_DEL  . . . . . . . . . . . . .  	NUMBER	007F	
C_ETB  . . . . . . . . . . . . .  	NUMBER	0017	
C_ETX  . . . . . . . . . . . . .  	NUMBER	0003	
C_HT . . . . . . . . . . . . . .  	NUMBER	0009	
C_LF . . . . . . . . . . . . . .  	NUMBER	000A	
C_NAK  . . . . . . . . . . . . .  	NUMBER	0015	

DAAMN  . . . . . . . . . . . . .  	L BYTE	049A	CONST	Global
DASMN  . . . . . . . . . . . . .  	L BYTE	049E	CONST	Global
DBCS . . . . . . . . . . . . . .  	NUMBER	0000	
DBMN . . . . . . . . . . . . . .  	L BYTE	0436	CONST	Global
DB_OPER  . . . . . . . . . . . .  	L NEAR	0000	CODE	External
DCINC_OPER . . . . . . . . . . .  	L NEAR	0000	CODE	External
DEALLOC  . . . . . . . . . . . .  	NUMBER	0049	
Microsoft (R) Macro Assembler Version 5.10                  2/14/25 23:44:19
DEBCONST.ASM                                                Symbols-7


DEBUG  . . . . . . . . . . . . .  	NUMBER	0000	
DECMN  . . . . . . . . . . . . .  	L BYTE	04A2	CONST	Global
DEVID_BLOCK_DEV  . . . . . . . .  	NUMBER	001F	
DEVID_DEVICE . . . . . . . . . .  	NUMBER	0080	
DEVID_DEVICE_CLOCK . . . . . . .  	NUMBER	0008	
DEVID_DEVICE_CON_IN  . . . . . .  	NUMBER	0001	
DEVID_DEVICE_CON_OUT . . . . . .  	NUMBER	0002	
DEVID_DEVICE_EOF . . . . . . . .  	NUMBER	0040	
DEVID_DEVICE_NULL  . . . . . . .  	NUMBER	0004	
DEVID_DEVICE_RAW . . . . . . . .  	NUMBER	0020	
DEVID_DEVICE_SPECIAL . . . . . .  	NUMBER	0010	
DEVID_EOF  . . . . . . . . . . .  	NUMBER	0040	
DEVID_FILE_CLEAN . . . . . . . .  	NUMBER	0040	
DEVID_FILE_MASK_DRIVE  . . . . .  	NUMBER	003F	
DEVID_ISCIN  . . . . . . . . . .  	NUMBER	0001	
DEVID_ISCLK  . . . . . . . . . .  	NUMBER	0008	
DEVID_ISCOT  . . . . . . . . . .  	NUMBER	0002	
DEVID_ISDEV  . . . . . . . . . .  	NUMBER	0080	
DEVID_ISNUL  . . . . . . . . . .  	NUMBER	0004	
DEVID_RAW  . . . . . . . . . . .  	NUMBER	0020	
DEVID_SPECIAL  . . . . . . . . .  	NUMBER	0010	
DIMN . . . . . . . . . . . . . .  	L BYTE	047E	CONST	Global
DIREG  . . . . . . . . . . . . .  	NUMBER	4944	
DIRSTRLEN  . . . . . . . . . . .  	NUMBER	0043	
DIR_SEARCH_FIRST . . . . . . . .  	NUMBER	0011	
DIR_SEARCH_NEXT  . . . . . . . .  	NUMBER	0012	
DISAVE . . . . . . . . . . . . .  	L WORD	0D93	CONST	Global
DISK_RESET . . . . . . . . . . .  	NUMBER	000D	
DISP8_OPER . . . . . . . . . . .  	L NEAR	0000	CODE	External
DISPB  . . . . . . . . . . . . .  	L WORD	0DA7	CONST	Global
DISTAB . . . . . . . . . . . . .  	L WORD	0036	CONST	Global
DIVMN  . . . . . . . . . . . . .  	L BYTE	04A6	CONST	Global
DOORG  . . . . . . . . . . . . .  	L NEAR	0000	CODE	External
DOUBLE_QUOTE . . . . . . . . . .  	NUMBER	0022	
DOWNMN . . . . . . . . . . . . .  	L BYTE	07BA	CONST	Global
DPBSIZ . . . . . . . . . . . . .  	NUMBER	0021	
DSIZ . . . . . . . . . . . . . .  	L BYTE	0DA5	CONST	Global
DSKSIZ . . . . . . . . . . . . .  	NUMBER	000D	
DSPRE  . . . . . . . . . . . . .  	L NEAR	0000	CODE	External
DSSAVE . . . . . . . . . . . . .  	L WORD	0D95	CONST	Global
DSSEGMN  . . . . . . . . . . . .  	L BYTE	07EE	CONST	Global
DUP_PDB  . . . . . . . . . . . .  	NUMBER	0055	
DW_OPER  . . . . . . . . . . . .  	L NEAR	0000	CODE	External
DXSAVE . . . . . . . . . . . . .  	L WORD	0D8B	CONST	Global

ECS_CALL . . . . . . . . . . . .  	NUMBER	0063	
EIMN . . . . . . . . . . . . . .  	L BYTE	07BE	CONST	Global
EMS_GET_MAN_STAT . . . . . . . .  	NUMBER	0040	
EMS_GET_PAGE_MAP . . . . . . . .  	NUMBER	0000	
EMS_GET_SET_PG_MP  . . . . . . .  	NUMBER	004E	
EMS_HANDLE_CNT . . . . . . . . .  	NUMBER	004B	
EMS_HANDLE_PAGES . . . . . . . .  	NUMBER	004D	
EMS_HANDLE_TOTAL . . . . . . . .  	NUMBER	00FF	
EMS_HAN_ALLOC  . . . . . . . . .  	NUMBER	0043	
EMS_LIM_40 . . . . . . . . . . .  	NUMBER	0040	
EMS_MAP_BUFF_SIZE  . . . . . . .  	NUMBER	000C	
EMS_MAP_MEMORY . . . . . . . . .  	NUMBER	0044	
EMS_PAGE_DEALL . . . . . . . . .  	NUMBER	0045	
EMS_PG_FRAME . . . . . . . . . .  	NUMBER	5800	
EMS_REST_PAGE_MAP  . . . . . . .  	NUMBER	0048	
EMS_SAVE_PAGE_MAP  . . . . . . .  	NUMBER	0047	
EMS_SET_PAGE_MAP . . . . . . . .  	NUMBER	0001	
EMS_UNALL_PG_CNT . . . . . . . .  	NUMBER	0042	
EMS_VERSION  . . . . . . . . . .  	NUMBER	0046	
ENTRYPOINT . . . . . . . . . . .  	NUMBER	00C0	
ERRACT_ABORT . . . . . . . . . .  	NUMBER	0004	
ERRACT_DLYRET  . . . . . . . . .  	NUMBER	0002	
ERRACT_IGNORE  . . . . . . . . .  	NUMBER	0006	
ERRACT_INTRET  . . . . . . . . .  	NUMBER	0007	
ERRACT_PANIC . . . . . . . . . .  	NUMBER	0005	
ERRACT_RETRY . . . . . . . . . .  	NUMBER	0001	
ERRACT_USER  . . . . . . . . . .  	NUMBER	0003	
ERRCLASS_ALREADY . . . . . . . .  	NUMBER	000C	
ERRCLASS_APPERR  . . . . . . . .  	NUMBER	0007	
ERRCLASS_AUTH  . . . . . . . . .  	NUMBER	0003	
ERRCLASS_BADFMT  . . . . . . . .  	NUMBER	0009	
Microsoft (R) Macro Assembler Version 5.10                  2/14/25 23:44:19
DEBCONST.ASM                                                Symbols-8


ERRCLASS_HRDFAIL . . . . . . . .  	NUMBER	0005	
ERRCLASS_INTRN . . . . . . . . .  	NUMBER	0004	
ERRCLASS_LOCKED  . . . . . . . .  	NUMBER	000A	
ERRCLASS_MEDIA . . . . . . . . .  	NUMBER	000B	
ERRCLASS_NOTFND  . . . . . . . .  	NUMBER	0008	
ERRCLASS_OUTRES  . . . . . . . .  	NUMBER	0001	
ERRCLASS_SYSFAIL . . . . . . . .  	NUMBER	0006	
ERRCLASS_TEMPSIT . . . . . . . .  	NUMBER	0002	
ERRCLASS_UNK . . . . . . . . . .  	NUMBER	000D	
ERRLOC_DISK  . . . . . . . . . .  	NUMBER	0002	
ERRLOC_MEM . . . . . . . . . . .  	NUMBER	0005	
ERRLOC_NET . . . . . . . . . . .  	NUMBER	0003	
ERRLOC_SERDEV  . . . . . . . . .  	NUMBER	0004	
ERRLOC_UNK . . . . . . . . . . .  	NUMBER	0001	
ERROR_ACCESS_DENIED  . . . . . .  	NUMBER	0005	
ERROR_ALREADY_ASSIGNED . . . . .  	NUMBER	0055	
ERROR_ARENA_TRASHED  . . . . . .  	NUMBER	0007	
ERROR_BAD_COMMAND  . . . . . . .  	NUMBER	0016	
ERROR_BAD_ENVIRONMENT  . . . . .  	NUMBER	000A	
ERROR_BAD_FORMAT . . . . . . . .  	NUMBER	000B	
ERROR_BAD_LENGTH . . . . . . . .  	NUMBER	0018	
ERROR_BAD_UNIT . . . . . . . . .  	NUMBER	0014	
ERROR_CANNOT_MAKE  . . . . . . .  	NUMBER	0052	
ERROR_CODE_PAGE_MISMATCHED . . .  	NUMBER	0025	
ERROR_CRC  . . . . . . . . . . .  	NUMBER	0017	
ERROR_CURRENT_DIRECTORY  . . . .  	NUMBER	0010	
ERROR_DUP_FCB  . . . . . . . . .  	NUMBER	0051	
ERROR_FAIL_I24 . . . . . . . . .  	NUMBER	0053	
ERROR_FCB_UNAVAILABLE  . . . . .  	NUMBER	0023	
ERROR_FILE_EXISTS  . . . . . . .  	NUMBER	0050	
ERROR_FILE_NOT_FOUND . . . . . .  	NUMBER	0002	
ERROR_GEN_FAILURE  . . . . . . .  	NUMBER	001F	
ERROR_HANDLE_DISK_FULL . . . . .  	NUMBER	0027	
ERROR_HANDLE_EOF . . . . . . . .  	NUMBER	0026	
ERROR_I24_BAD_COMMAND  . . . . .  	NUMBER	0003	
ERROR_I24_BAD_LENGTH . . . . . .  	NUMBER	0005	
ERROR_I24_BAD_UNIT . . . . . . .  	NUMBER	0001	
ERROR_I24_CRC  . . . . . . . . .  	NUMBER	0004	
ERROR_I24_GEN_FAILURE  . . . . .  	NUMBER	000C	
ERROR_I24_NOT_DOS_DISK . . . . .  	NUMBER	0007	
ERROR_I24_NOT_READY  . . . . . .  	NUMBER	0002	
ERROR_I24_OUT_OF_PAPER . . . . .  	NUMBER	0009	
ERROR_I24_READ_FAULT . . . . . .  	NUMBER	000B	
ERROR_I24_SECTOR_NOT_FOUND . . .  	NUMBER	0008	
ERROR_I24_SEEK . . . . . . . . .  	NUMBER	0006	
ERROR_I24_WRITE_FAULT  . . . . .  	NUMBER	000A	
ERROR_I24_WRITE_PROTECT  . . . .  	NUMBER	0000	
ERROR_I24_WRONG_DISK . . . . . .  	NUMBER	000F	
ERROR_INVALID_ACCESS . . . . . .  	NUMBER	000C	
ERROR_INVALID_BLOCK  . . . . . .  	NUMBER	0009	
ERROR_INVALID_DATA . . . . . . .  	NUMBER	000D	
ERROR_INVALID_DRIVE  . . . . . .  	NUMBER	000F	
ERROR_INVALID_FUNCTION . . . . .  	NUMBER	0001	
ERROR_INVALID_HANDLE . . . . . .  	NUMBER	0006	
ERROR_INVALID_PARAMETER  . . . .  	NUMBER	0057	
ERROR_INVALID_PASSWORD . . . . .  	NUMBER	0056	
ERROR_LOCK_VIOLATION . . . . . .  	NUMBER	0021	
ERROR_NET_WRITE_FAULT  . . . . .  	NUMBER	0058	
ERROR_NOT_DOS_DISK . . . . . . .  	NUMBER	001A	
ERROR_NOT_ENOUGH_MEMORY  . . . .  	NUMBER	0008	
ERROR_NOT_READY  . . . . . . . .  	NUMBER	0015	
ERROR_NOT_SAME_DEVICE  . . . . .  	NUMBER	0011	
ERROR_NOT_SUPPORTED  . . . . . .  	NUMBER	0032	
ERROR_NO_MORE_FILES  . . . . . .  	NUMBER	0012	
ERROR_OUT_OF_PAPER . . . . . . .  	NUMBER	001C	
ERROR_OUT_OF_STRUCTURES  . . . .  	NUMBER	0054	
ERROR_PATH_NOT_FOUND . . . . . .  	NUMBER	0003	
ERROR_READ_FAULT . . . . . . . .  	NUMBER	001E	
ERROR_SECTOR_NOT_FOUND . . . . .  	NUMBER	001B	
ERROR_SEEK . . . . . . . . . . .  	NUMBER	0019	
ERROR_SHARING_BUFFER_EXCEEDED  .  	NUMBER	0024	
ERROR_SHARING_VIOLATION  . . . .  	NUMBER	0020	
ERROR_SYS_COMP_NOT_LOADED  . . .  	NUMBER	005A	
ERROR_TOO_MANY_OPEN_FILES  . . .  	NUMBER	0004	
ERROR_WRITE_FAULT  . . . . . . .  	NUMBER	001D	
ERROR_WRITE_PROTECT  . . . . . .  	NUMBER	0013	
Microsoft (R) Macro Assembler Version 5.10                  2/14/25 23:44:19
DEBCONST.ASM                                                Symbols-9


ERROR_WRONG_DISK . . . . . . . .  	NUMBER	0022	
ESCMN  . . . . . . . . . . . . .  	L BYTE	04AA	CONST	Global
ESC_OPER . . . . . . . . . . . .  	L NEAR	0000	CODE	External
ESPRE  . . . . . . . . . . . . .  	L NEAR	0000	CODE	External
ESSAVE . . . . . . . . . . . . .  	L WORD	0D97	CONST	Global
ESSEGMN  . . . . . . . . . . . .  	L BYTE	07E2	CONST	Global
EXEC . . . . . . . . . . . . . .  	NUMBER	004B	
EXEC_BLOCK . . . . . . . . . . .  	L BYTE	0E0A	CONST	Global
EXEC_FUNC_NO_EXECUTE . . . . . .  	NUMBER	0001	
EXEC_FUNC_OVERLAY  . . . . . . .  	NUMBER	0002	
EXEFCB . . . . . . . . . . . . .  	ALIAS	 FCB		
EXE_VALID_OLD_SIGNATURE  . . . .  	NUMBER	4D5A	
EXE_VALID_SIGNATURE  . . . . . .  	NUMBER	5A4D	
EXISTS_MASK  . . . . . . . . . .  	NUMBER	000F	
EXIT . . . . . . . . . . . . . .  	NUMBER	004C	
EXIT_ABORT . . . . . . . . . . .  	NUMBER	0000	
EXIT_CTRL_C  . . . . . . . . . .  	NUMBER	0001	
EXIT_HARD_ERROR  . . . . . . . .  	NUMBER	0002	
EXIT_KEEP_PROCESS  . . . . . . .  	NUMBER	0003	
EXIT_TERMINATE . . . . . . . . .  	NUMBER	0000	
EXPECTED_VERSION . . . . . . . .  	NUMBER	0004	
EXTHANDLE  . . . . . . . . . . .  	NUMBER	0067	
EXTOPEN  . . . . . . . . . . . .  	NUMBER	006C	
EXT_EXISTS_FAIL  . . . . . . . .  	NUMBER	0000	
EXT_EXISTS_OPEN  . . . . . . . .  	NUMBER	0001	
EXT_FILE_NOT_EXISTS  . . . . . .  	NUMBER	0004	
EXT_NEXISTS_CREATE . . . . . . .  	NUMBER	0010	
EXT_OPEN_I24_OFF . . . . . . . .  	NUMBER	0002	
EXT_OPEN_ON  . . . . . . . . . .  	NUMBER	0001	
EX_OPER  . . . . . . . . . . . .  	L NEAR	0000	CODE	External

FALSE  . . . . . . . . . . . . .  	NUMBER	0000	
FCB  . . . . . . . . . . . . . .  	NUMBER	005C	
FCBDEVICE  . . . . . . . . . . .  	NUMBER	0040	
FCBMASK  . . . . . . . . . . . .  	NUMBER	00C0	
FCBNETWORK . . . . . . . . . . .  	NUMBER	0080	
FCBSHARE . . . . . . . . . . . .  	NUMBER	00C0	
FCBSPECIAL . . . . . . . . . . .  	NUMBER	0080	
FCB_CLOSE  . . . . . . . . . . .  	NUMBER	0010	
FCB_CREATE . . . . . . . . . . .  	NUMBER	0016	
FCB_DELETE . . . . . . . . . . .  	NUMBER	0013	
FCB_L_ATTR . . . . . . . . . . .  	BYTE	001E	
FCB_L_DRIVE  . . . . . . . . . .  	BYTE	0019	
FCB_L_FIRCLUS  . . . . . . . . .  	WORD	001A	
FCB_L_MFS  . . . . . . . . . . .  	WORD	001C	
FCB_NETID  . . . . . . . . . . .  	DWORD	001C	
FCB_NET_DRIVE  . . . . . . . . .  	BYTE	0019	
FCB_NET_HANDLE . . . . . . . . .  	WORD	001A	
FCB_NSLD_DRIVE . . . . . . . . .  	BYTE	0019	
FCB_NSLD_DRVPTR  . . . . . . . .  	DWORD	001A	
FCB_NSL_BITS . . . . . . . . . .  	BYTE	001A	
FCB_NSL_DIRPOS . . . . . . . . .  	BYTE	001F	
FCB_NSL_DIRSEC . . . . . . . . .  	WORD	001D	
FCB_NSL_DRIVE  . . . . . . . . .  	BYTE	0019	
FCB_NSL_FIRCLUS  . . . . . . . .  	WORD	001B	
FCB_OPEN . . . . . . . . . . . .  	NUMBER	000F	
FCB_RANDOM_READ  . . . . . . . .  	NUMBER	0021	
FCB_RANDOM_READ_BLOCK  . . . . .  	NUMBER	0027	
FCB_RANDOM_WRITE . . . . . . . .  	NUMBER	0022	
FCB_RANDOM_WRITE_BLOCK . . . . .  	NUMBER	0028	
FCB_RENAME . . . . . . . . . . .  	NUMBER	0017	
FCB_SEQ_READ . . . . . . . . . .  	NUMBER	0014	
FCB_SEQ_WRITE  . . . . . . . . .  	NUMBER	0015	
FCB_SFN  . . . . . . . . . . . .  	BYTE	0018	
FCHK . . . . . . . . . . . . . .  	NUMBER	0001	
FD9_OPER . . . . . . . . . . . .  	L NEAR	0000	CODE	External
FDB_OPER . . . . . . . . . . . .  	L NEAR	0000	CODE	External
FDELIM . . . . . . . . . . . . .  	NUMBER	0002	
FDE_OPER . . . . . . . . . . . .  	L NEAR	0000	CODE	External
FFCB . . . . . . . . . . . . . .  	NUMBER	0008	
FGROUP . . . . . . . . . . . . .  	L NEAR	0000	CODE	External
FGROUP3  . . . . . . . . . . . .  	L NEAR	0000	CODE	External
FGROUP3W . . . . . . . . . . . .  	L NEAR	0000	CODE	External
FGROUPB  . . . . . . . . . . . .  	L NEAR	0000	CODE	External
FGROUPDS . . . . . . . . . . . .  	L NEAR	0000	CODE	External
FGROUPP  . . . . . . . . . . . .  	L NEAR	0000	CODE	External
Microsoft (R) Macro Assembler Version 5.10                  2/14/25 23:44:19
DEBCONST.ASM                                                Symbols-10


FGROUPX  . . . . . . . . . . . .  	L NEAR	0000	CODE	External
FGROUPZ  . . . . . . . . . . . .  	L NEAR	0000	CODE	External
FILDIRENT  . . . . . . . . . . .  	NUMBER	0010	
FILE_TIMES . . . . . . . . . . .  	NUMBER	0057	
FILPERPROC . . . . . . . . . . .  	NUMBER	0014	
FIND_FIRST . . . . . . . . . . .  	NUMBER	004E	
FIND_NEXT  . . . . . . . . . . .  	NUMBER	004F	
FI_TAB . . . . . . . . . . . . .  	L BYTE	0819	CONST	Global
FLAGTAB  . . . . . . . . . . . .  	L WORD	0C45	CONST	Global
FLSAVE . . . . . . . . . . . . .  	L WORD	0D9F	CONST	Global
FSPCHK . . . . . . . . . . . . .  	NUMBER	0004	
F_AUX  . . . . . . . . . . . . .  	NUMBER	0010	
F_CARRY  . . . . . . . . . . . .  	NUMBER	0001	
F_DIRECTION  . . . . . . . . . .  	NUMBER	0400	
F_INTERRUPT  . . . . . . . . . .  	NUMBER	0200	
F_OVERFLOW . . . . . . . . . . .  	NUMBER	0800	
F_PARITY . . . . . . . . . . . .  	NUMBER	0004	
F_SIGN . . . . . . . . . . . . .  	NUMBER	0080	
F_TRACE  . . . . . . . . . . . .  	NUMBER	0100	
F_ZERO . . . . . . . . . . . . .  	NUMBER	0040	

GENERIC_IOCTL  . . . . . . . . .  	NUMBER	440D	
GETADDR  . . . . . . . . . . . .  	L NEAR	0000	CODE	External
GETCURRENTPSP  . . . . . . . . .  	NUMBER	0062	
GETEXTCNTRY  . . . . . . . . . .  	NUMBER	0065	
GETEXTENDEDERROR . . . . . . . .  	NUMBER	0059	
GETSETCDPG . . . . . . . . . . .  	NUMBER	0066	
GETSETMEDIAID  . . . . . . . . .  	NUMBER	0069	
GET_CURRENT_PDB  . . . . . . . .  	NUMBER	0051	
GET_DATA16 . . . . . . . . . . .  	L NEAR	0000	CODE	External
GET_DATE . . . . . . . . . . . .  	NUMBER	002A	
GET_DEFAULT_DPB  . . . . . . . .  	NUMBER	001F	
GET_DEFAULT_DRIVE  . . . . . . .  	NUMBER	0019	
GET_DMA  . . . . . . . . . . . .  	NUMBER	002F	
GET_DPB  . . . . . . . . . . . .  	NUMBER	0032	
GET_DRIVE_FREESPACE  . . . . . .  	NUMBER	0036	
GET_FCB_FILE_LENGTH  . . . . . .  	NUMBER	0023	
GET_FCB_POSITION . . . . . . . .  	NUMBER	0024	
GET_INDOS_FLAG . . . . . . . . .  	NUMBER	0034	
GET_INTERRUPT_VECTOR . . . . . .  	NUMBER	0035	
GET_IN_VARS  . . . . . . . . . .  	NUMBER	0052	
GET_TIME . . . . . . . . . . . .  	NUMBER	002C	
GET_VERIFY_ON_WRITE  . . . . . .  	NUMBER	0054	
GET_VERSION  . . . . . . . . . .  	NUMBER	0030	
GROUP1 . . . . . . . . . . . . .  	L NEAR	0000	CODE	External
GROUP2 . . . . . . . . . . . . .  	L NEAR	0000	CODE	External
GRP1 . . . . . . . . . . . . . .  	L NEAR	0000	CODE	External
GRP1TAB  . . . . . . . . . . . .  	L WORD	0BF3	CONST	Global
GRP2 . . . . . . . . . . . . . .  	L NEAR	0000	CODE	External
GRP2TAB  . . . . . . . . . . . .  	L WORD	0C03	CONST	Global

HANDLE_FAIL_I24  . . . . . . . .  	NUMBER	0100	
HEADSAVE . . . . . . . . . . . .  	L WORD	0E08	CONST	Global
HLTMN  . . . . . . . . . . . . .  	L BYTE	064F	CONST	Global
HONGEUL  . . . . . . . . . . . .  	NUMBER	0063	

I24_AREA . . . . . . . . . . . .  	NUMBER	0006	
I24_CLASS  . . . . . . . . . . .  	NUMBER	0080	
I24_OPERATION  . . . . . . . . .  	NUMBER	0001	
IBM  . . . . . . . . . . . . . .  	ALIAS	 IBMVER		
IBMCOPYRIGHT . . . . . . . . . .  	ALIAS	 FALSE		
IBMJAPAN . . . . . . . . . . . .  	ALIAS	 FALSE		
IBMJAPVER  . . . . . . . . . . .  	ALIAS	 FALSE		
IBMVER . . . . . . . . . . . . .  	ALIAS	 TRUE		
IDIVMN . . . . . . . . . . . . .  	L BYTE	0653	CONST	Global
IFS_IOCTL  . . . . . . . . . . .  	NUMBER	006B	
IMMED  . . . . . . . . . . . . .  	L NEAR	0000	CODE	External
IMMTAB . . . . . . . . . . . . .  	L WORD	0BE3	CONST	Global
IMULMN . . . . . . . . . . . . .  	L BYTE	0658	CONST	Global
INCMN  . . . . . . . . . . . . .  	L BYTE	065D	CONST	Global
INFIXB . . . . . . . . . . . . .  	L NEAR	0000	CODE	External
INFIXW . . . . . . . . . . . . .  	L NEAR	0000	CODE	External
INMN . . . . . . . . . . . . . .  	L BYTE	066A	CONST	Global
INSTALLED  . . . . . . . . . . .  	NUMBER	FFFF	
INSTALLEDDATA  . . . . . . . . .  	NUMBER	0000	
INT3 . . . . . . . . . . . . . .  	L NEAR	0000	CODE	External
Microsoft (R) Macro Assembler Version 5.10                  2/14/25 23:44:19
DEBCONST.ASM                                                Symbols-11


INTBASE  . . . . . . . . . . . .  	NUMBER	0080	
INTERNAT . . . . . . . . . . . .  	ALIAS	 FALSE		
INTERNATIONAL  . . . . . . . . .  	NUMBER	0038	
INTERNAT_BLOCK_MAX . . . . . . .  	NUMBER	0020	
INTMN  . . . . . . . . . . . . .  	L BYTE	0666	CONST	Global
INTOMN . . . . . . . . . . . . .  	L BYTE	0661	CONST	Global
INTTAB . . . . . . . . . . . . .  	NUMBER	0020	
INT_24_ERROR . . . . . . . . . .  	NUMBER	2000	
INT_ABORT  . . . . . . . . . . .  	ALIAS	 INTTAB		
INT_COMMAND  . . . . . . . . . .  	NUMBER	0021	
INT_CTRL_C . . . . . . . . . . .  	NUMBER	0023	
INT_DISK_READ  . . . . . . . . .  	NUMBER	0025	
INT_DISK_WRITE . . . . . . . . .  	NUMBER	0026	
INT_FASTCON  . . . . . . . . . .  	NUMBER	0029	
INT_FATAL_ABORT  . . . . . . . .  	NUMBER	0024	
INT_IBM  . . . . . . . . . . . .  	NUMBER	002A	
INT_KEEP_PROCESS . . . . . . . .  	NUMBER	0027	
INT_MASK . . . . . . . . . . . .  	NUMBER	00FF	
INT_OPER . . . . . . . . . . . .  	L NEAR	0000	CODE	External
INT_SPOOLER  . . . . . . . . . .  	NUMBER	0028	
INT_TERMINATE  . . . . . . . . .  	NUMBER	0022	
INVARB . . . . . . . . . . . . .  	L NEAR	0000	CODE	External
INVARW . . . . . . . . . . . . .  	L NEAR	0000	CODE	External
IN_OPER  . . . . . . . . . . . .  	L NEAR	0000	CODE	External
IOCTL  . . . . . . . . . . . . .  	NUMBER	0044	
IO_MODE_ID . . . . . . . . . . .  	NUMBER	0002	
IPSAVE . . . . . . . . . . . . .  	L WORD	0D9D	CONST	Global
IRETMN . . . . . . . . . . . . .  	L BYTE	066D	CONST	Global

JAMN . . . . . . . . . . . . . .  	L BYTE	067B	CONST	Global
JAPAN  . . . . . . . . . . . . .  	ALIAS	 FALSE		
JBEMN  . . . . . . . . . . . . .  	L BYTE	0687	CONST	Global
JCMN . . . . . . . . . . . . . .  	L BYTE	068B	CONST
JCXZMN . . . . . . . . . . . . .  	L BYTE	067E	CONST	Global
JGEMN  . . . . . . . . . . . . .  	L BYTE	06A4	CONST	Global
JGMN . . . . . . . . . . . . . .  	L BYTE	06A8	CONST	Global
JLEMN  . . . . . . . . . . . . .  	L BYTE	06B4	CONST	Global
JLMN . . . . . . . . . . . . . .  	L BYTE	06B8	CONST	Global
JMPCALL  . . . . . . . . . . . .  	L NEAR	0000	CODE	External
JMPMN  . . . . . . . . . . . . .  	L BYTE	06C4	CONST	Global
JMP_OPER . . . . . . . . . . . .  	L NEAR	0000	CODE	External
JNCMN  . . . . . . . . . . . . .  	L BYTE	0683	CONST	Global
JNOMN  . . . . . . . . . . . . .  	L BYTE	06E0	CONST	Global
JNSMN  . . . . . . . . . . . . .  	L BYTE	06DC	CONST	Global
JNZMN  . . . . . . . . . . . . .  	L BYTE	06C8	CONST	Global
JOMN . . . . . . . . . . . . . .  	L BYTE	06E4	CONST	Global
JPEMN  . . . . . . . . . . . . .  	L BYTE	06D0	CONST	Global
JPOMN  . . . . . . . . . . . . .  	L BYTE	06D4	CONST	Global
JSMN . . . . . . . . . . . . . .  	L BYTE	06E7	CONST	Global
JZMN . . . . . . . . . . . . . .  	L BYTE	069E	CONST	Global

KANJI  . . . . . . . . . . . . .  	ALIAS	 FALSE		
KEEP_PROCESS . . . . . . . . . .  	NUMBER	0031	
KOREA  . . . . . . . . . . . . .  	ALIAS	 FALSE		

LAHFMN . . . . . . . . . . . . .  	L BYTE	06ED	CONST	Global
LBUFFCNT . . . . . . . . . . . .  	L BYTE	0DAA	CONST	Global
LBUFSIZ  . . . . . . . . . . . .  	L BYTE	0DA9	CONST	Global
LDSMN  . . . . . . . . . . . . .  	L BYTE	06F2	CONST	Global
LEAMN  . . . . . . . . . . . . .  	L BYTE	06F6	CONST	Global
LESMN  . . . . . . . . . . . . .  	L BYTE	06FA	CONST	Global
LF . . . . . . . . . . . . . . .  	NUMBER	000A	
LINEBUF  . . . . . . . . . . . .  	L BYTE	0DAB	CONST	Global
LOADACC  . . . . . . . . . . . .  	L NEAR	0000	CODE	External
LOCKMN . . . . . . . . . . . . .  	L BYTE	06FE	CONST	Global
LOCKOPER . . . . . . . . . . . .  	NUMBER	005C	
LODBMN . . . . . . . . . . . . .  	L BYTE	0703	CONST	Global
LODWMN . . . . . . . . . . . . .  	L BYTE	0709	CONST	Global
LONGJMP  . . . . . . . . . . . .  	L NEAR	0000	CODE	External
LOOPMN . . . . . . . . . . . . .  	L BYTE	0729	CONST	Global
LOOPNZMN . . . . . . . . . . . .  	L BYTE	070F	CONST	Global
LOOPZMN  . . . . . . . . . . . .  	L BYTE	0716	CONST	Global
LOWER_A  . . . . . . . . . . . .  	NUMBER	0061	
LOWER_Z  . . . . . . . . . . . .  	NUMBER	007A	
LSEEK  . . . . . . . . . . . . .  	NUMBER	0042	
LSEEK_EOF_OPTION . . . . . . . .  	NUMBER	0002	
Microsoft (R) Macro Assembler Version 5.10                  2/14/25 23:44:19
DEBCONST.ASM                                                Symbols-12


LSEEK_FROM_START . . . . . . . .  	NUMBER	0000	
L_OPER . . . . . . . . . . . . .  	L NEAR	0000	CODE	External

M8087  . . . . . . . . . . . . .  	L NEAR	0000	CODE	External
M8087_D9 . . . . . . . . . . . .  	L NEAR	0000	CODE	External
M8087_DB . . . . . . . . . . . .  	L NEAR	0000	CODE	External
M8087_DD . . . . . . . . . . . .  	L NEAR	0000	CODE	External
M8087_DF . . . . . . . . . . . .  	L NEAR	0000	CODE	External
M8087_TAB  . . . . . . . . . . .  	L BYTE	07F6	CONST	Global
MAJOR_VERSION  . . . . . . . . .  	NUMBER	0004	
MASK_PORT  . . . . . . . . . . .  	NUMBER	0021	
MAXBUCKETINPAGE  . . . . . . . .  	NUMBER	0002	
MAXBUFFINBUCKET  . . . . . . . .  	NUMBER	000F	
MAXOP  . . . . . . . . . . . . .  	NUMBER	00C1		Global
MD9_TAB  . . . . . . . . . . . .  	L BYTE	0863	CONST	Global
MD9_TAB2 . . . . . . . . . . . .  	L BYTE	0885	CONST	Global
MDB_TAB  . . . . . . . . . . . .  	L BYTE	0914	CONST	Global
MDB_TAB2 . . . . . . . . . . . .  	L BYTE	092E	CONST	Global
MDD_TAB  . . . . . . . . . . . .  	L BYTE	0941	CONST	Global
MDD_TAB2 . . . . . . . . . . . .  	L BYTE	095F	CONST	Global
MDF_TAB  . . . . . . . . . . . .  	L BYTE	096F	CONST	Global
MEMIMM . . . . . . . . . . . . .  	L NEAR	0000	CODE	External
MEMS . . . . . . . . . . . . . .  	NUMBER	0001	
MINOR_VERSION  . . . . . . . . .  	NUMBER	0000	
MI_INT . . . . . . . . . . . . .  	NUMBER	00CD	
MI_LONG_CALL . . . . . . . . . .  	NUMBER	009A	
MI_LONG_JMP  . . . . . . . . . .  	NUMBER	00EA	
MI_LONG_RET  . . . . . . . . . .  	NUMBER	00CB	
MI_NEAR_RET  . . . . . . . . . .  	NUMBER	00C3	
MKDIR  . . . . . . . . . . . . .  	NUMBER	0039	
MOVBMN . . . . . . . . . . . . .  	L BYTE	072E	CONST	Global
MOVMN  . . . . . . . . . . . . .  	L BYTE	073A	CONST	Global
MOVSEGFROM . . . . . . . . . . .  	L NEAR	0000	CODE	External
MOVSEGTO . . . . . . . . . . . .  	L NEAR	0000	CODE	External
MOVWMN . . . . . . . . . . . . .  	L BYTE	0734	CONST	Global
MOV_OPER . . . . . . . . . . . .  	L NEAR	0000	CODE	External
MSVER  . . . . . . . . . . . . .  	NUMBER	0000	
MULMN  . . . . . . . . . . . . .  	L BYTE	073E	CONST	Global
MULTDOS  . . . . . . . . . . . .  	NUMBER	0012	
MULTIFS  . . . . . . . . . . . .  	NUMBER	0011	
MULTNET  . . . . . . . . . . . .  	NUMBER	0011	
MULTSHARE  . . . . . . . . . . .  	NUMBER	0010	

NAMESPEC . . . . . . . . . . . .  	L BYTE	0DA2	CONST	Global
NEGMN  . . . . . . . . . . . . .  	L BYTE	0742	CONST	Global
NEWEXEC  . . . . . . . . . . . .  	L BYTE	0DFF	CONST	Global
NEXTCS . . . . . . . . . . . . .  	L WORD	0E04	CONST	Global
NEXTIP . . . . . . . . . . . . .  	L WORD	0E06	CONST	Global
NLSFUNC  . . . . . . . . . . . .  	NUMBER	0014	
NOOPERANDS . . . . . . . . . . .  	L NEAR	0000	CODE	External
NOPMN  . . . . . . . . . . . . .  	L BYTE	0746	CONST	Global
NOREGL . . . . . . . . . . . . .  	L BYTE	0DA6	CONST	Global
NOTMN  . . . . . . . . . . . . .  	L BYTE	074A	CONST	Global
NOT_EXISTS_MASK  . . . . . . . .  	NUMBER	00F0	
NO_CODE_PAGE_CHECK . . . . . . .  	NUMBER	0100	
NO_OPER  . . . . . . . . . . . .  	L NEAR	0000	CODE	External

OEM_C1 . . . . . . . . . . . . .  	NUMBER	00F9	
OEM_C2 . . . . . . . . . . . . .  	NUMBER	00FA	
OEM_C3 . . . . . . . . . . . . .  	NUMBER	00FB	
OEM_C4 . . . . . . . . . . . . .  	NUMBER	00FC	
OEM_C5 . . . . . . . . . . . . .  	NUMBER	00FD	
OEM_C6 . . . . . . . . . . . . .  	NUMBER	00FE	
OEM_C7 . . . . . . . . . . . . .  	NUMBER	00FF	
OPBUFLEN . . . . . . . . . . . .  	NUMBER	0023	
OPEN . . . . . . . . . . . . . .  	NUMBER	003D	
OPEN_FOR_BOTH  . . . . . . . . .  	NUMBER	0002	
OPEN_FOR_READ  . . . . . . . . .  	NUMBER	0000	
OPEN_FOR_WRITE . . . . . . . . .  	NUMBER	0001	
OPTAB  . . . . . . . . . . . . .  	L BYTE	0990	CONST	Global
ORGMN  . . . . . . . . . . . . .  	L BYTE	043E	CONST
ORMN . . . . . . . . . . . . . .  	L BYTE	0456	CONST	Global
OUTFIXB  . . . . . . . . . . . .  	L NEAR	0000	CODE	External
OUTFIXW  . . . . . . . . . . . .  	L NEAR	0000	CODE	External
OUTMN  . . . . . . . . . . . . .  	L BYTE	074E	CONST	Global
OUTVARB  . . . . . . . . . . . .  	L NEAR	0000	CODE	External
Microsoft (R) Macro Assembler Version 5.10                  2/14/25 23:44:19
DEBCONST.ASM                                                Symbols-13


OUTVARW  . . . . . . . . . . . .  	L NEAR	0000	CODE	External
OUT_OPER . . . . . . . . . . . .  	L NEAR	0000	CODE	External

PARSE_FILE_DESCRIPTOR  . . . . .  	NUMBER	0029	
PATHPARSE  . . . . . . . . . . .  	NUMBER	0061	
PDB_APPEND . . . . . . . . . . .  	BYTE	003D	
PDB_INTERCON . . . . . . . . . .  	BYTE	003C	
PFLAG  . . . . . . . . . . . . .  	L BYTE	0DFC	CONST	Global
POPFMN . . . . . . . . . . . . .  	L BYTE	0752	CONST	Global
POPMN  . . . . . . . . . . . . .  	L BYTE	0757	CONST	Global
POP_OPER . . . . . . . . . . . .  	L NEAR	0000	CODE	External
PREFIX . . . . . . . . . . . . .  	L NEAR	0000	CODE	External
PROMPT . . . . . . . . . . . . .  	NUMBER	002D	
PUSHFMN  . . . . . . . . . . . .  	L BYTE	075B	CONST	Global
PUSHMN . . . . . . . . . . . . .  	L BYTE	0761	CONST	Global
PUSH_OPER  . . . . . . . . . . .  	L NEAR	0000	CODE	External

QFLAG  . . . . . . . . . . . . .  	L BYTE	0DFE	CONST	Global

RAW_CON_INPUT  . . . . . . . . .  	NUMBER	0007	
RAW_CON_IO . . . . . . . . . . .  	NUMBER	0006	
RCLMN  . . . . . . . . . . . . .  	L BYTE	0766	CONST	Global
RCRMN  . . . . . . . . . . . . .  	L BYTE	076A	CONST	Global
RDFLG  . . . . . . . . . . . . .  	L BYTE	0DA3	CONST	Global
READ . . . . . . . . . . . . . .  	NUMBER	003F	
READ_SECTOR  . . . . . . . . . .  	NUMBER	0000	
READ_WRITE . . . . . . . . . . .  	NUMBER	0008	
REDIRECTOR . . . . . . . . . . .  	NUMBER	0000	
REG16  . . . . . . . . . . . . .  	L BYTE	0010	CONST	Global
REG8 . . . . . . . . . . . . . .  	L BYTE	0000	CONST	Global
REGDIF . . . . . . . . . . . . .  	NUMBER	016A		Global
REGIMMB  . . . . . . . . . . . .  	L NEAR	0000	CODE	External
REGIMMW  . . . . . . . . . . . .  	L NEAR	0000	CODE	External
REGOP  . . . . . . . . . . . . .  	L NEAR	0000	CODE	External
REGTAB . . . . . . . . . . . . .  	L BYTE	0C1B	CONST	Global
REGTABEND  . . . . . . . . . . .  	L WORD	0C45	CONST	Global
REGTABLEN  . . . . . . . . . . .  	NUMBER	000E	
RENAME . . . . . . . . . . . . .  	NUMBER	0056	
REPNZMN  . . . . . . . . . . . .  	L BYTE	0773	CONST	Global
REPZMN . . . . . . . . . . . . .  	L BYTE	076E	CONST	Global
RESERVED_BITS_MASK . . . . . . .  	NUMBER	FE00	
RETFMN . . . . . . . . . . . . .  	L BYTE	0788	CONST	Global
RETMN  . . . . . . . . . . . . .  	L BYTE	078D	CONST	Global
RETSAVE  . . . . . . . . . . . .  	L WORD	0E00	CONST	Global
RMDIR  . . . . . . . . . . . . .  	NUMBER	003A	
ROLMN  . . . . . . . . . . . . .  	L BYTE	0791	CONST	Global
RORMN  . . . . . . . . . . . . .  	L BYTE	0795	CONST	Global
ROTOP  . . . . . . . . . . . . .  	L NEAR	0000	CODE	External
RSETFLAG . . . . . . . . . . . .  	L BYTE	0DA1	CONST	Global
RSTACK . . . . . . . . . . . . .  	L WORD	0D99	CONST	Global

SAHFMN . . . . . . . . . . . . .  	L BYTE	0799	CONST	Global
SARMN  . . . . . . . . . . . . .  	L BYTE	079E	CONST	Global
SAV16  . . . . . . . . . . . . .  	L NEAR	0000	CODE	External
SAV8 . . . . . . . . . . . . . .  	L NEAR	0000	CODE	External
SAVHEX . . . . . . . . . . . . .  	L NEAR	0000	CODE	External
SBBMN  . . . . . . . . . . . . .  	L BYTE	044E	CONST	Global
SCABMN . . . . . . . . . . . . .  	L BYTE	07A2	CONST	Global
SCAWMN . . . . . . . . . . . . .  	L BYTE	07A8	CONST	Global
SEGDIF . . . . . . . . . . . . .  	NUMBER	0000	
SEGOP  . . . . . . . . . . . . .  	L NEAR	0000	CODE	External
SEGTAB . . . . . . . . . . . . .  	L WORD	0C13	CONST	Global
SERVERCALL . . . . . . . . . . .  	NUMBER	005D	
SETBLOCK . . . . . . . . . . . .  	NUMBER	004A	
SETCNTC  . . . . . . . . . . . .  	ALIAS	 TRUE		
SETDPB . . . . . . . . . . . . .  	NUMBER	0053	
SET_CTRL_C_TRAPPING  . . . . . .  	NUMBER	0033	
SET_CURRENT_PDB  . . . . . . . .  	NUMBER	0050	
SET_DATE . . . . . . . . . . . .  	NUMBER	002B	
SET_DEFAULT_DRIVE  . . . . . . .  	NUMBER	000E	
SET_DMA  . . . . . . . . . . . .  	NUMBER	001A	
SET_DRIVEID_OPTION . . . . . . .  	NUMBER	0001	
SET_INTERRUPT_VECTOR . . . . . .  	NUMBER	0025	
SET_OEM_HANDLER  . . . . . . . .  	NUMBER	00F8	
SET_PRINTER_FLAG . . . . . . . .  	NUMBER	0064	
SET_TIME . . . . . . . . . . . .  	NUMBER	002D	
Microsoft (R) Macro Assembler Version 5.10                  2/14/25 23:44:19
DEBCONST.ASM                                                Symbols-14


SET_VERIFY_ON_WRITE  . . . . . .  	NUMBER	002E	
SF_BUSY  . . . . . . . . . . . .  	NUMBER	-0001	
SF_CLOSE_NODATE  . . . . . . . .  	NUMBER	4000	
SF_DEFAULT_NUMBER  . . . . . . .  	NUMBER	0005	
SF_FSDA  . . . . . . . . . . . .  	BYTE	0019	
SF_ISFCB . . . . . . . . . . . .  	NUMBER	8000	
SF_ISNET . . . . . . . . . . . .  	NUMBER	8000	
SF_LRU . . . . . . . . . . . . .  	WORD	0015	
SF_NETID . . . . . . . . . . . .  	BYTE	0019	
SF_NET_SPOOL . . . . . . . . . .  	NUMBER	0800	
SF_NO_INHERIT  . . . . . . . . .  	NUMBER	1000	
SF_OPENAGE . . . . . . . . . . .  	WORD	0017	
SF_PIPE  . . . . . . . . . . . .  	NUMBER	2000	
SF_SERIAL_ID . . . . . . . . . .  	WORD	000B	
SHAREF . . . . . . . . . . . . .  	NUMBER	0000	
SHARING_COMPAT . . . . . . . . .  	NUMBER	0000	
SHARING_DENY_BOTH  . . . . . . .  	NUMBER	0010	
SHARING_DENY_NONE  . . . . . . .  	NUMBER	0040	
SHARING_DENY_READ  . . . . . . .  	NUMBER	0030	
SHARING_DENY_WRITE . . . . . . .  	NUMBER	0020	
SHARING_MASK . . . . . . . . . .  	NUMBER	00F0	
SHARING_NET_FCB  . . . . . . . .  	NUMBER	0070	
SHARING_NO_INHERIT . . . . . . .  	NUMBER	0080	
SHFTAB . . . . . . . . . . . . .  	L WORD	0BD3	CONST	Global
SHIFT  . . . . . . . . . . . . .  	L NEAR	0000	CODE	External
SHIFTV . . . . . . . . . . . . .  	L NEAR	0000	CODE	External
SHLMN  . . . . . . . . . . . . .  	L BYTE	07AE	CONST	Global
SHORTJMP . . . . . . . . . . . .  	L NEAR	0000	CODE	External
SHRMN  . . . . . . . . . . . . .  	L BYTE	07B2	CONST	Global
SIGNIMM  . . . . . . . . . . . .  	L NEAR	0000	CODE	External
SINGLE_QUOTE . . . . . . . . . .  	NUMBER	0027	
SIREG  . . . . . . . . . . . . .  	NUMBER	4953	
SISAVE . . . . . . . . . . . . .  	L WORD	0D91	CONST	Global
SIZ8 . . . . . . . . . . . . . .  	L BYTE	002A	CONST	Global
SIZE_TAB . . . . . . . . . . . .  	L BYTE	0823	CONST	Global
SPSAVE . . . . . . . . . . . . .  	L WORD	0D8D	CONST	Global
SREG . . . . . . . . . . . . . .  	L BYTE	0020	CONST	Global
SSPRE  . . . . . . . . . . . . .  	L NEAR	0000	CODE	External
SSSAVE . . . . . . . . . . . . .  	L WORD	0D99	CONST	Global
SSSEGMN  . . . . . . . . . . . .  	L BYTE	07EA	CONST	Global
STACK  . . . . . . . . . . . . .  	L BYTE	0D85	CONST	Global
STCMN  . . . . . . . . . . . . .  	L BYTE	07B6	CONST	Global
STDAUX . . . . . . . . . . . . .  	NUMBER	0003	
STDERR . . . . . . . . . . . . .  	NUMBER	0002	
STDIN  . . . . . . . . . . . . .  	NUMBER	0000	
STDOUT . . . . . . . . . . . . .  	NUMBER	0001	
STDPRN . . . . . . . . . . . . .  	NUMBER	0004	
STD_AUX_INPUT  . . . . . . . . .  	NUMBER	0003	
STD_AUX_OUTPUT . . . . . . . . .  	NUMBER	0004	
STD_CON_INPUT  . . . . . . . . .  	NUMBER	0001	
STD_CON_INPUT_FLUSH  . . . . . .  	NUMBER	000C	
STD_CON_INPUT_NO_ECHO  . . . . .  	NUMBER	0008	
STD_CON_INPUT_STATUS . . . . . .  	NUMBER	000B	
STD_CON_OUTPUT . . . . . . . . .  	NUMBER	0002	
STD_CON_STRING_INPUT . . . . . .  	NUMBER	000A	
STD_CON_STRING_OUTPUT  . . . . .  	NUMBER	0009	
STD_PRINTER_OUTPUT . . . . . . .  	NUMBER	0005	
STOBMN . . . . . . . . . . . . .  	L BYTE	07C2	CONST	Global
STOREACC . . . . . . . . . . . .  	L NEAR	0000	CODE	External
STOWMN . . . . . . . . . . . . .  	L BYTE	07C8	CONST	Global
SUBMN  . . . . . . . . . . . . .  	L BYTE	044A	CONST	Global
SYSVER . . . . . . . . . . . . .  	ALIAS	 FALSE		

TEMPLEN  . . . . . . . . . . . .  	NUMBER	0086	
TESTMN . . . . . . . . . . . . .  	L BYTE	07CE	CONST	Global
TOTREG . . . . . . . . . . . . .  	L BYTE	0DA4	CONST	Global
TRUE . . . . . . . . . . . . . .  	NUMBER	FFFF	
TRUEBYTE . . . . . . . . . . . .  	NUMBER	00FF	
TST_OPER . . . . . . . . . . . .  	L NEAR	0000	CODE	External

UNLINK . . . . . . . . . . . . .  	NUMBER	0041	
UPMN . . . . . . . . . . . . . .  	L BYTE	047A	CONST	Global
UPPER_A  . . . . . . . . . . . .  	NUMBER	0041	
UPPER_C  . . . . . . . . . . . .  	NUMBER	0043	
UPPER_E  . . . . . . . . . . . .  	NUMBER	0045	
UPPER_F  . . . . . . . . . . . .  	NUMBER	0046	
Microsoft (R) Macro Assembler Version 5.10                  2/14/25 23:44:19
DEBCONST.ASM                                                Symbols-15


UPPER_L  . . . . . . . . . . . .  	NUMBER	004C	
UPPER_M  . . . . . . . . . . . .  	NUMBER	004D	
UPPER_N  . . . . . . . . . . . .  	NUMBER	004E	
UPPER_P  . . . . . . . . . . . .  	NUMBER	0050	
UPPER_S  . . . . . . . . . . . .  	NUMBER	0053	
UPPER_X  . . . . . . . . . . . .  	NUMBER	0058	
UPPER_Z  . . . . . . . . . . . .  	NUMBER	005A	
USEROPER . . . . . . . . . . . .  	NUMBER	005E	
USER_PROC_PDB  . . . . . . . . .  	L WORD	0E02	CONST	Global

VEC_BREAKPOINT . . . . . . . . .  	NUMBER	0003	
VEC_CRIT_ERR . . . . . . . . . .  	NUMBER	0024	
VEC_CTRL_BREAK . . . . . . . . .  	NUMBER	0023	
VEC_PRIMITIVE_DISK_READ  . . . .  	NUMBER	0025	
VEC_PRIMITIVE_DISK_WRITE . . . .  	NUMBER	0026	
VEC_SING_STEP  . . . . . . . . .  	NUMBER	0001	
VEC_TERM_ADDR  . . . . . . . . .  	NUMBER	0022	

WAITMN . . . . . . . . . . . . .  	L BYTE	07D3	CONST	Global
WAITPROCESS  . . . . . . . . . .  	NUMBER	004D	
WORDTOALU  . . . . . . . . . . .  	L NEAR	0000	CODE	External
WRITE  . . . . . . . . . . . . .  	NUMBER	0040	
WRITE_SECTOR . . . . . . . . . .  	NUMBER	0000	

XCHGAX . . . . . . . . . . . . .  	L NEAR	0000	CODE	External
XCHGMN . . . . . . . . . . . . .  	L BYTE	07D8	CONST	Global
XDUP . . . . . . . . . . . . . .  	NUMBER	0045	
XDUP2  . . . . . . . . . . . . .  	NUMBER	0046	
XLATMN . . . . . . . . . . . . .  	L BYTE	07DD	CONST	Global
XM_ERR80 . . . . . . . . . . . .  	NUMBER	0080	
XM_ERR83 . . . . . . . . . . . .  	NUMBER	0083	
XM_ERR84 . . . . . . . . . . . .  	NUMBER	0084	
XM_ERR85 . . . . . . . . . . . .  	NUMBER	0085	
XM_ERR86 . . . . . . . . . . . .  	NUMBER	0086	
XM_ERR87 . . . . . . . . . . . .  	NUMBER	0087	
XM_ERR88 . . . . . . . . . . . .  	NUMBER	0088	
XM_ERR89 . . . . . . . . . . . .  	NUMBER	0089	
XM_ERR8A . . . . . . . . . . . .  	NUMBER	008A	
XM_ERR8B . . . . . . . . . . . .  	NUMBER	008B	
XM_ERR8D . . . . . . . . . . . .  	NUMBER	008D	
XM_ERR8E . . . . . . . . . . . .  	NUMBER	008E	
XM_ERR8F . . . . . . . . . . . .  	NUMBER	008F	
XM_NOT_INST  . . . . . . . . . .  	NUMBER	00FF	
XNAMETRANS . . . . . . . . . . .  	NUMBER	0060	
XORMN  . . . . . . . . . . . . .  	L BYTE	0452	CONST	Global

ZZOPCODE . . . . . . . . . . . .  	L BYTE	0BD3	CONST

?PLM . . . . . . . . . . . . . .  	NUMBER	0000	
?WIN . . . . . . . . . . . . . .  	NUMBER	0000	
@CPU . . . . . . . . . . . . . .  	TEXT  0101h		
@FILENAME  . . . . . . . . . . .  	TEXT  debconst		
@VERSION . . . . . . . . . . . .  	TEXT  510		


   3724 Source  Lines
   3836 Total   Lines
   1100 Symbols

  41388 + 162324 Bytes symbol space free

      0 Warning Errors
      0 Severe  Errors
